:020000020000FC
:0200000050C1ED
:02000800567828
:100034000C942F300C942D300C94E61C0C94F21D6F
:1000440078C17EC188C18CC1C8EDD1E00895C4E1F6
:10005400D1E00895C0E0D1E00895CCE3DDE0089557
:10006400E0E0F6EF0895E0E0F6EF0895C8E8D1E0A7
:100074000895CEE2DDE00895FF91FF93EF2FE85459
:10008400F2E4FA5FE650E8F7EE2726F4EA0FFB1FE6
:10009400EE0FFF1F08956894EFCFE894EDCF0C9412
:1000A400F4320C9419330C9425330C947C320C9454
:1000B40009330C94FC370C94C43A0C94BC3A0C9459
:1000C40003330C9406330C94B9330C9435340C94E8
:1000D40049330C94A4330C94E8350C94C7350C9430
:1000E400CF35E8940C94123768940C9412370C941E
:1000F400243E0C94FC330C94503D0E94E8350C943F
:100104002F380C9421380C942838409120014F71D9
:100114000895409139010895409122010895409134
:10012400230108950C946C390C9485390C94C039CE
:100134000C9478390C9495390C94D7390C94A538CF
:100144000C94CD3E0C94AA3E0C9452390C945F3915
:100154000C94A0390C9441390C94FD350C94D4378B
:100164000C9459370C9472370E9411190C944C3C1E
:100174000E9411190C94813C0C94373C0C943E3C25
:100184000C94453C0C94E6390C94393A0C94B63CE6
:100194000C94F33C0C94B13C0C94EE3C0C948537D9
:1001A4000C94B1370C9404380C94AB3A0C94E03EA4
:1001B4000C94FC3E0C94003F0C94403F0C94533F31
:1001C4000C940E3F0C940A3F0C94143F0C94193F6A
:1001D4000C94103F0C945E3F0C94803F0C94893F28
:1001E4000C94D80C0C94F10C0C94F00C0C94FC0CA6
:1001F4000C945A0D0C94250D0C94280D0C947B0D25
:100204000C94820D0C948A0D0C949B0D0C94AB0DE4
:100214000C94270E0C943A0F0C94F7410C945B4207
:100224000C94CC420C9472420C948F410C94CA3FAF
:100234000C9471410E9452420C94274088270E94DA
:10024400F33F0C94EF4088270E94B9400C940F4070
:100254000C94F70D0C94FA0E0C94DD3A0C94C93AF4
:100264000C94FE0F0C94330B0C94C71D0C940D1CB2
:100274000C94211C0C9457280C941C280C94587929
:100284000F900F900C94F12A5BD00C94E033AF9351
:10029400BF930C9474340C94F5350C940536F8948F
:1002A400A0E02A2EA1E03A2EA0E1AEBFAFEFADBF91
:1002B4000E94F3310E94033F0E940B790E944C3A42
:1002C400ECECFF27408155EA508350814083A09194
:1002D4003501AF7E553A21F4B0911801B5FFA06104
:1002E400A09335010E94B933AFEFA0931001A093FE
:1002F4003D0120924901AA270E947C3220925C0190
:100304008827789420923901209222010C94C1010B
:1003140042954A9540934901A7E00E94F432AA27E6
:100324000E9425330E94B9330E94CE040E942138D2
:10033400B6CFAF91BF91CF91DF91EF91FF91089527
:100344000F901F90FF93EF93DF93CF93BF93AF93DF
:100354001F920F9208957F916F915F914F91E9CF12
:100364000F901F90FF93EF93DF93CF93BF93AF93BF
:100374004F935F936F937F931F920F920895A1E021
:100384000E942533AA270E947C329927A7E10E9464
:10039400F4320E94B933A0E10E94F432C4E0DAE0FE
:1003A400E7E3F7E10E947237A7E00E94F4320E946B
:1003B400CF35070420001DD1A6E10E94F432C5E028
:1003C400D8E0E6E0F9E00E947237D8E1F9E10E9452
:1003D4007237D8E0F9E0CC5FEC5FC833A0F364EB8C
:1003E4000E94FC374091200141FD0DC04091230142
:1003F400403011F00C9424026A9591F74091650104
:100404004077C1F385CF0E94B9330E94CF350000F5
:100414004B6579626F6172642D54657374000E9438
:10042400FC3370917101A0917101A215E1F3209246
:10043400710190E07A2F0E94A4330E943434F3CFE8
:100444000E942838A0E00E942533A1E00E944A3986
:10045400992720923601AA270E947C32A7E00E94A5
:10046400F4320E94B933A5E10E94F432C0E0D0E036
:10047400EDE1F4E10E94B137A1E50E94F4320E945B
:10048400CF350101838383838383204156522D43D7
:1004940068697042617369633220828282828282D7
:1004A4000000C9EAD4E00AE408830B8F04EC098352
:1004B4000A8F0CE80A83098F08E20B83088F02E68F
:1004C4000C830F8B06EA0D830E8B47D1D8D2409153
:1004D40049014B3008F0442740934901642F67FDDC
:1004E40066276B3008F06AE020E06F9397D06F9135
:1004F40023952830D1F796D16BD105D16F93BCD118
:100504006F91423E11F46A95EACF433E11F463952C
:10051400E6CF443E21F4643010F06450E0CF453E11
:1005240021F4673010F46C5FDACF6830E0F04A3EB3
:1005340011F0443F19F760934901683031F44A3EA1
:10054400E9F667D00E94C7207BCF693031F44A3E78
:10055400A9F65FD00E94C72573CF5BD04A3E71F6DF
:100564000E9476276DCF4F934091200142FD20C019
:100574004F914A3E11F0443F29F449D088270E9404
:10058400CE045ECF413F29F442D088270E94B104B3
:1005940057CF423F21F43BD00E94752251CF433FB5
:1005A40031F435D00E94DC220E941E0B49CFA6CF25
:1005B4004F91413F21F42BD00E94540441CF423F3C
:1005C40031F425D00E946A250E941A2839CF433F6E
:1005D40041F41DD00E946A250E9455280E941E0BDA
:1005E4002FCF443F21F713D00E949E040E941E0B7C
:1005F40027CF0E94CF35FF4156522D436869704280
:1006040061736963322056312E3235000895609348
:100614004901A0912201A030E1F70895A1E0B3E0DF
:1006240020FDA95F21FDA25F22FDBA5F422F0E9437
:100634009779042F4EE20E3421F44CE25F3F09F027
:100644004AE2621709F44295409338010E94E83562
:100654000E94CF35FF20200040E50E943534422F10
:100664004F5C0E9435340E94CF35FF202000B395A3
:100674000E94E835422F0E9497794E34B1F4709667
:10068400BA950E94E83513E004E00E9434344591A1
:100694000E9435340A95D9F70E943434B3950E94E8
:1006A400E8351A9589F7BA950FC00E94CF35FF2017
:1006B40020D0D1202000B3950E94E8350E94CF3588
:1006C400FF2020D2D3202000422F0E94127AB3951B
:1006D4000E94E83566E045910E9435346A95D9F761
:1006E400B3950E94E83566E045910E9435346A95D9
:1006F400D9F7B3950E94E8350E94CF35FF2020201A
:100704002020200008954AE26A3009F4429540937B
:1007140038010E94CF350F0F202020202020000018
:100724000E94CF35100F2020D4D5202000000E9435
:10073400CF35110F2020D6D7202000000E94CF35BE
:10074400120F20494E464F2000000E94CF35130F50
:10075400202020202020000008954AE24093380100
:100764000E94CF3510154D43553A36343400ECEC25
:10077400FF27408125EA208320814083253A19F40C
:1007840040E50E9435340E94CF3512154B42443A5D
:100794000000E0E0F9E844910E943534E0584491C7
:1007A4000E9435340E94CF3511155649443A000051
:1007B4007091350172FD06C00E94CF35FF4E54532F
:1007C400430005C00E94CF35FF50414C20000895DE
:1007D40048E2693009F44295409338010E94CF35CC
:1007E4000F0820202020202000000E94CF35100870
:1007F4002020D8D9202000000E94CF3511082020C5
:10080400DADB202000000E94CF351208434F4E4609
:10081400494700000E94CF351308202020202020C3
:10082400000008954CE2683009F442954093380181
:100834000E94CF350F0120202020202000000E949C
:10084400CF3510012020DCDD202000000E94CF35B0
:1008540011012020DEDF202000000E94CF3512018C
:1008640044464C41534800000E94CF3513012020D8
:1008740020202020000008953DED209223010E94B5
:10088400BD38409120014470431739F0342F403073
:1008940011F4F5D0F4CFF8D0F2CF409123014030D9
:1008A40071F30895A4E00E94F432C1E0DFE0ECE1CA
:1008B400F3E10E94B137A0E40E94F4320E941E0BBF
:1008C4000E94CF351002436F70792050726F6772A7
:1008D400616D20746F007091490160E0ACE06717AE
:1008E40009F4A0E60E94F432B2E1A62FAA0FA60FE3
:1008F400AD5F0E94E83540E50E943534462F4770CD
:100904004F5C0E9435346395683041F70E9421386A
:10091400423E21F47030D1F37A95DFCF433E21F487
:100924007730A1F37395D9CF4A3E19F40E94417AE6
:1009340008954D3E59F708950E94EE3C4F436C656F
:10094400617220746869732050726F6772616D3FC1
:100954002000413009F008950E941B7A08950E94F6
:1009640028380E9495794E3441F00E94C80520929F
:100974003901A0912301A43F09F064CD0E94957927
:1009840044914F3561F308D00E940B790E944C3A90
:10099400AA270E947C32E3CF0E94B9338827209291
:1009A40022010E94107A44914F3561F03C964591A2
:1009B4004E3449F47396F695E79509950E940B79A0
:1009C4000E944C3A08950E94970F0E940B790E944E
:1009D4004C3A2092190120925C01209236010E9427
:1009E400C43A0E94FC330E94F432A0E4A0930001B4
:1009F400A0EEA0930101A0914A01A770A03019F4C0
:100A0400A7E2B6E127C0A130B1F4A7E20E94F43214
:100A1400C0E0DDE0E8E0FEE0E8940E941237A2E7DF
:100A24000E94F432C0E0D8E6E7E4F3E70E947237AC
:100A3400A7E2B9E60FC0A23019F4A0E1B2E40AC0FB
:100A4400A33019F4A0E1BFE205C0A53089F4A0E108
:100A5400B8E300C00E94F432AA270E94E8350E943D
:100A6400CF35FF20505245535320455343200000B7
:100A7400A0912201AD3EE1F70E9428380895E2E9F1
:100A8400FAE00E94393A0895E0EBFAE0FACF202028
:100A9400202020202045646974202053617665203D
:100AA400204C6F6164202052756E2020202020206D
:100AB400202020436F7079202053656E64202052DB
:100AC4006563762020436C656172AA270E942533F2
:100AD400A3E00E944A398F93409149010E941479FE
:100AE4000E94B9330E94713299274091220140300B
:100AF400E1F70E94CF3500002050524F4752414D3C
:100B04002000409149014F5C0E9435344AE30E9421
:100B14003534C3EED1E050D2F0D20E94DF79E8D36D
:100B24008F91A8E8803069F1ACECE4E2F3E1813024
:100B340031F0ABE48A9545914030E9F7F8CF44D2DF
:100B440092E0A5E0B1E00E94E8350E94C7350E941A
:100B5400CF35FF20494E20500000409146014F5CA4
:100B64000E9435344AE30E943534BB27AC2DA3954B
:100B74000E9449334AE30E943534AD2DA3950E9467
:100B840049330895AAE25A2E70E208959927FADFAC
:100B94009CDF32D5D0923A010E9448380E94BD3879
:100BA40050912001403E21F4AA2752FDBB2733C0B7
:100BB400413E31F4AFE152FDAA2752FDBEE52BC000
:100BC400423E11F4AA9527C0433E69F4A3959B2F96
:100BD4000E94EC0A9A1730F4BE3511F4AA951BC092
:100BE400AA27B39518C0443E21F4BA95B7FDBB2794
:100BF40012C0463E21F4B850B7FDBB270CC0473E97
:100C040011F4B85F08C0453E11F4B39504C04A3EE0
:100C140039F5B395AA27A03838F0AFE1BA95B038C2
:100C2400C0F0AA27BB27B6CFA03228F0BE3589F082
:100C3400AA27B395AFCFBF3508F0BEE50B2F0D152E
:100C440008F4D02E0D2D015F0B1718F40B2F0F5045
:100C5400D02E9B2F0E94EC0A9A1708F4A92F9ACF42
:100C64009B2F4E3E39F4AF93BF930E94B80ABF91B5
:100C7400AF916AC14F3E31F4BF930E94C30ABF9142
:100C8400AA2762C1493E11F474D15EC14C3E31F4CD
:100C9400A03009F481CFAA956CD156C1547009F4DF
:100CA400ABC0433FD9F4ACEC8FD10E94CF350107E0
:100CB400524543454956452050524F4752414D20D5
:100CC400592F4E203F0061D136F468D211D35ADF38
:100CD400B3D45092D80170D188275BCF423F39F505
:100CE400ACEC72D10E94CF35010753454E442050DD
:100CF400524F4752414D20592F4E203F000045D1BD
:100D040056F7ACEC61D10E94CF35010753454E44F0
:100D1400494E472E2E2E2020202020202020000067
:100D24003092360186D1209236012CDFD4CF443F55
:100D3400C1F4ACEC49D10E94CF350107434C454185
:100D4400522050524F4752414D20592F4E203F00C0
:100D54001CD136F4BFD2CCD215DF6ED45092D80158
:100D6400BACF413F41F5ACEC2FD10E94CF350107FA
:100D74005052494E542050524F4752414D20592F02
:100D84004E203F0002D1B6F4ABE41ED10E94CF3511
:100D940001075052494E54494E472E2E2E202020F2
:100DA400202020202000A2E0A093360142D12092EE
:100DB4003601E8DE90CF433611F45DD2EDCE4837EC
:100DC40031F40E943D0976D25092D80113C0C5EF88
:100DD400D1E0463779F46881623469F460E269935A
:100DE4006993699369936993699338D281D25092D4
:100DF400D801D2CE8827D0CE423F11F5BF93AF930E
:100E0400D7D0D9F0ACECE0D00E94CF3501075341E4
:100E140056452050524F4752414D20592F4E203FA6
:100E24000000B3D046F40E94A4790E94DF7960D216
:100E3400A9DE7093D801C0D08827AF91BF91AACE04
:100E4400433FE1F4BF93AF93B3D0B9F0ACECBCD063
:100E54000E94CF3501074C4F5354204348414E471D
:100E6400455320592F4E203F00008FD026F70E9473
:100E7400DF793ED287DE7093D801DDCF413F49F45C
:100E84006A2E7B2EBBD0A62DB72D5092D80184CECE
:100E9400D2CF4D3E11F5BF93AF938AD0A9F0ACECFD
:100EA40093D00E94CF3501075155495420572F4FF5
:100EB400205341564520592F4E203F0066D046F717
:100EC400A0912201A030E1F70E946932A0E00E94C3
:100ED4007C32AF91BF91A5D30895443FE9F4A1D3E7
:100EE40067D029F40E9469320E94B9330895A9E6B3
:100EF4006BD00E94CF3501075341564520434841EA
:100F04004E474553204245464F52452052554E21A7
:100F140000000E9421388FCF4B3E59F4A93148F488
:100F240040E215D040E2EA2FE35071F0E8F70FD029
:100F3400F9CF5091200152FD09C053FD07C04C3137
:100F440028F0403818F403D05092D80125CEAF31A0
:100F540061F05A2FAFE10E949C386A916983AA9587
:100F6400A517D9F74883A39508950E949C38488310
:100F740008950E949C385A2F5F3121F0498149938A
:100F84005395FACF50E2588308950E942138493589
:100F940059F0493749F04A3E39F04E3439F04E366B
:100FA40029F04D3E19F0F1CF68940895E89408951E
:100FB400A091D801A0320895A8E806D00E94CF35A8
:100FC40001054F4B00000895EF93FF939927A093D9
:100FD4004C010E94CF350105202020202020202014
:100FE40020202020202020202020202020202020FD
:100FF400202020202000FF91EF910895A0E00E947E
:1010040070384A3E09F40895423E21F4A030B9F301
:10101400AA95F5CF433E21F4AB3089F3A395EFCFE6
:10102400403268F3403858F74883AB3009F0A39551
:10103400E6CFC9EDD1E057E049910E9435345A9585
:10104400D9F756E122965CE049910E9435345A95CD
:10105400D9F70E94FC334EE511D016F04A95E1F71A
:10106400542F53954427451719F024D04395FBCFAB
:1010740043E20E9435340E94FC330895CF93DF93FA
:101084005F936F93E894C4E4D2E053E2459FC00DAC
:10109400D11D50E26991613238F45A95D9F76F91B4
:1010A4005F91DF91CF91089568946F915F91DF9183
:1010B400CF910895DF93CF934F935F936F93C1E4E0
:1010C400D2E053E2459FC00DD11DDF93CF93A39689
:1010D40053E26A91613210F45A95D9F7CF91DF91B6
:1010E40049910E9435345A95D9F70E94FC336F9187
:1010F4005F914F91CF91DF9108950E94A2014F9388
:10110400ECE1F1E1AEE1B2E04591403011F04D93F4
:10111400FBCF4F910C949B012045786974202020CB
:101124004E616D6520202053617665202052656CE8
:101134006F616420202052756E2020000E94A2015D
:101144004F93ECE4F1E1DECF20202020202020206A
:101154005072696E74202053656E6420202052659D
:101164006376202020204E65772020000E94A20173
:101174004F93ECE7F1E1C6CF2041626F72742020F7
:10118400202020202020202020202020202020205B
:10119400202020202020202020202000E7DFACEC8D
:1011A40013DF0E94CF350105524543454956494E48
:1011B400472E2E2E000020923A018CD099D09927E8
:1011C400ECECE0934C01E3EEF1E0EE2EFF2E41E176
:1011D4000E946C395CE00E94C0394B31B9F14A334A
:1011E400D1F70E94C0394B3189F1403218F0419354
:1011F4005A95B9F7403228F00E94C0394B3131F189
:10120400F9CFEEE1F2E0EE2EFF2E53E2EE2DFF2DAC
:10121400B396EE2EFF2E0E94C0394B31B9F0403206
:10122400D0F3433299F006C00E94C0394B3171F0BB
:10123400403248F041935A95B9F70E94C0394B3176
:1012440029F04032D0F793959036F9F60895A3E249
:10125400BA9FA1E4B2E0A00DB11D0895BF93AF936E
:10126400F6DFC8E8D1E053E249914D935A95E1F78E
:10127400AF91BF910895BF93AF93C5EFD1E0A2E4BE
:10128400A993A5E5A993A6E4A993ADE3A993DFDF08
:10129400C8E8D1E053E24D9149935A95E1F7409162
:1012A40088014093F901409189014093FA01AF917B
:1012B400BF910895BF93AF934F935F93C8DF139685
:1012C40040E250E24D935A95E9F75F914F91AF9107
:1012D400BF9108950E94A2014F9340E2A1E4B2E0BD
:1012E400CDEFDCE04D932197E9F74F910C949B01EE
:1012F4000E94A2014F9341E0A1E4B2E0C0E3D42FE5
:10130400DA5010F0C395FCCFD65CCD93DD93C0E2E8
:10131400CD9390964395403689F74F910C949B0159
:10132400425245414B004F564552464C4F5700449C
:101334004956494445202F30005351522046524FBC
:101344004D203C3000434F4E5354414E5420544F93
:101354004F204249470057524F4E4720455850525C
:10136400455353494F4E0053594E5441582045520A
:10137400524F5200554E4B4E4F574E204B455957E6
:101384004F52440057524F4E4720464F524D4154FE
:1013940000424144204C494E454E554D4245520071
:1013A4004E45585420572F4F20464F520052455413
:1013B40055524E20572F4F20474F535542005354F8
:1013C40041434B204F564552464C4F5700554E54BF
:1013D400494C20572F4F2052455045415400493223
:1013E40043204552524F5200554E4B4E4F574E20BC
:1013F4004552524F520044464C41534820455252A4
:101404004F52004F5554204F4620415252415900EB
:10141400494E434F4D504C45544520504152004B8A
:101424004559574F5244204953204D495353494E2F
:10143400470057524F4E472042434F505920004FC8
:101444005554204F462053435245454E0043414E88
:101454004E4F54204352454154452046494C450083
:101464004D454D4F52592046554C4C0046494C452C
:10147400204E4F5420464F554E440050414745207E
:101484004E4F5420494E2046494C45005041474553
:1014940053204E4F5420494E2052414E4745004E52
:1014A4004F5420494E204752415048494353204D00
:1014B4004F4445004E4F5420494E20544558542023
:1014C4004D4F4445004E4F205553522046494C45FC
:1014D40000535243204F5554204F46205343524506
:1014E400454E0044455354204F5554204F462053F5
:1014F400435245454E0057524F4E47205350524990
:1015040054450057524F4E4720454550524F4D20A9
:10151400414452004E4F205052472046494C45000A
:10152400584D4F44454D204552524F520043414E71
:1015340054204C4F4144205448495300494F2044BF
:10154400495341424C45440053455249414C312092
:101554004E4F5420415641494C41424C45004E4F58
:1015640020494F204452495645520000BE3508F0E8
:101574000895BF9323D0B395BE35E1F79BDEBF91A9
:10158400B7CEBE3508F00895BF93AF93AB2FAA959D
:10159400BDE508D0BA95BA17E1F7B3958BDEAF91E4
:1015A400BF91A6CE0E94A20152DE1396ED01B0E2D5
:1015B400A991AAA3BA95E1F70C949B010E94A201F8
:1015C40046DE1396ED01B0E2ABA1A993BA95E1F71B
:1015D4000C949B010E94A2013ADEED0193964E9178
:1015E4004132E8F34038D8F7AC1BBC0B9A2F925029
:1015F40097FD99270C949B012AD00E94803F4F3578
:1016040020F0AA27BB27D22C0895B42F0E94803F34
:101614004032B8F7A42F0E94803F403590F7D42E73
:10162400089515D04B2F0E94893F4A2F0E94893F6D
:101634004D2D0E94893F08950AD0422D0E94893F72
:10164400422D0E94893F422D0E94893F08950090B7
:101654004901C0EDD7E043E0409DC00DD11D089580
:101664002CC1CAEFDCE02A922A9280E02F92AA27AA
:10167400BB27442771917032E9F3703888F77A33C5
:1016840079F37E3709F041C07191733511F4D401B7
:1016940042C07C3421F4AC2DA395BB273CC07035EB
:1016A40029F4A0914601A395BB2735C0763539F4BA
:1016B400B0913501A9E3B2FFA7E0B1E02CC07835C1
:1016C40021F4A0915001BB2726C0793521F4A091C3
:1016D4005101BB2720C0723529F4A0912E0DB09181
:1016E4002F0D19C07E3421F4A0913A0DBB2713C0ED
:1016F4007D3439F460913501A1E064FDA2E0BB279B
:101704000AC07832F1F47CE112C07C3111F07E31F0
:1017140021F4A191BB27719122C07D3111F07F3159
:1017240021F4B191A19171911AC07C3160F4572FC9
:101734002E01EF015F93452FAA27BB27FE01E2018B
:1017440099CF87E0CAC0703398F07A3388F4403870
:1017540010F086E0C2C0A72FA053BB2771914F376A
:1017640009F426D1AA93BA9340E887CF85E0B5C09F
:101774007134A0F07B3590F4403810F086E0ADC0B1
:101784007154770FEF93FF93E0EAFCE0E70FF21D4B
:10179400A191B191FF91EF917191E1CF7D3251F41B
:1017A4004F3711F4442766CF20F4403210F04FE74E
:1017B40061CF59C0783231F471E07F93AA27BB27F7
:1017C400472F58CF793209F048C05F915D3188F5D1
:1017D400B991A991FF93EF93DF93CF9301E20F9314
:1017E4000CE00F930BEF1BE0050F121D0F931F93DB
:1017F400089586E00895DAC0E9C098C117C0A9C168
:1018040024C256C272C28EC295C293C295C278C215
:10181400DFC2CFC118C11AC1D3C1E7C1A5C1ACC1D0
:10182400B1C125C234C2E4C223C333C3B095A09569
:1018340008956AD0803009F050C0C7CF86E0000018
:10184400CF91DF91EF91FF91803009F00895AA9331
:10185400BA93AA27BB2742E00DCF4F3720F44F306D
:1018640010F086E03AC0608132E27C3339F46E33A2
:10187400C1F133E26D33A9F131E234C07E3329F48E
:1018840035E26D3371F134E22DC036E27D3351F12E
:1018940037E37B3239F138E37D3221F139E37332B6
:1018A40009F13AE47A32F1F03BE47F32D9F03CE4D6
:1018B4007532C1F03DE47632A9F05F91503021F0E9
:1018C4005F3130F021D0F9CFB991A99131970895C2
:1018D40086E05F915030C1F3FCCF4F914030E9F77F
:1018E40008953196732F5F91A72FB52FA07FB07FF6
:1018F400BA1720F009D0803081F7F5CF5F937F933A
:10190400AA27BB27472FB6CE5F934F93199109910E
:10191400B991A99127E9352F3F70330F330F230F66
:101924003CE0321D2F933F9308953BC0000000001C
:101934000000E6D036C000000000DBD0A150A1704A
:1019440030C0E6D0A150A1702CC0E2D02AC0000063
:101954000000D6D0A150A17024C0CBD022C000007A
:1019640000003DD01EC00000000038D01AC00000A6
:101974000000A02BB12B15C000003CD012C0000009
:10198400000096D00EC00000000092D0A22FB32F0A
:1019940008C0A023B12305C0000003C0000000005C
:1019A4000000AA93BA934F915F910895B7FF0895E9
:1019B400A095B09511960895AA93BA93089517FF28
:1019C400089500951095030D121D0895AB2B29F071
:1019D400B7FBA1E0BB270EF412970895F2DF2B2F7B
:1019E4002127A00FB11F27FD08952B2F212727FDA5
:1019F40082E008950BD0D901BF770EF4D9DF37FD0B
:101A040003C0452B09F4089582E008956DD0CEDF1C
:101A1400B19FA001A09F9001A19F300D411D521DB7
:101A2400B09F300D411D521D089508E611E0B038F5
:101A340018F0A00FB11FFBCFA017B10718F0A01B1F
:101A4400B10BFACF08950AE5A01BB209EEDFE8E175
:101A5400F6E80AE510E0A017B10738F4E00FF11F2B
:101A6400EA1BFB0BA491BB27089504EB10E0A0171D
:101A7400B10768F40AE510E0E01BF10BEA0FFB1F65
:101A8400A491BB27A095B095A30DB21D08950EE0B7
:101A940011E0A017B10728F4E00FF11FEA1BFB0BBC
:101AA400EFCF0EE011E0E01BF10BEA0FFB1FDACFE2
:101AB400212F202B11F483E0089516D022273327F9
:101AC400442751E1441FAA1FBB1F5A9551F0221FFE
:101AD400331F4FEF201B310BA8F7200F311F40E0BD
:101AE400F1CF0EF465CF08952B2F212727FB5EDF5E
:101AF40066CF0F931F930A271B27012B91F00FC06A
:101B04000F931F93B0581058A01BB10B50F007C08F
:101B14000F931F93B05810580A1B1B0B10F0AA27E1
:101B240001C0A1E0B0E01F910F91089584E0B7FDDA
:101B3400089588270A2F1B2FB2E0AA27232D3327C5
:101B4400021B130B20F0A3952B0F321DF9CFBB27DB
:101B540008954F935F938D010E945B3A59DFA42F40
:101B6400B52F5F914F910895AF3F11F0A0933F01BE
:101B7400A0913F01BB270895A0B90E94A61CA0B163
:101B8400BB27089510914A01103011F08CE108959B
:101B940004EC12E0A017B10710F082E10895FDE013
:101BA400ECE3EA0FFB1F68940E94E639A42FBB27DD
:101BB4000895B0937301A09372010E94AE1C08951E
:101BC400BF3F69F0A09378010E94A725803021F0DF
:101BD400AFEFBFEF88270895A42FBB2708950E9475
:101BE400AC258827B42FAA270895BF3FA1F4A0FDF0
:101BF40009C00E94A425803019F08827CC27DD274E
:101C0400DE0108950E94A425803019F08827EE276C
:101C1400FF27DF01F6CFA09378010E94A72580302B
:101C240021F08827AA27BB27ECCF7F9377270E9430
:101C3400AF25DF3F31F4CF3F21F4A72FBB277F919E
:101C4400E0CF7395703899F7F8CFA770A06CA09384
:101C54007C00A0917A00A064A0937A00A0917A00FD
:101C6400A6FDFCCFA0917800B09179000895BB3017
:101C740020F4BA3028F0A83C18F0AFEFBFEF089575
:101C8400C8EDD1E0CA0FDB1FA881BB270895B3308C
:101C940018F4B23010F0A7FD20CEDF93CF93CCE33D
:101CA400DDE0CA0FDB1F0E94AA3EA62FBB270895C2
:101CB400B43021F4BB27AC91BB270895B83040F071
:101CC4000E94361C40FF88E240FD0C940E72089579
:101CD400AF3F11F4A0B1F0CFA770A395B0B1B69502
:101CE400AA95E9F7AA27AA1FE7CF70916501777033
:101CF4000E94403FBB27A52F803009F08FE0089554
:101D0400ED01DC3040F40E94803FBB27A42F8030DB
:101D140009F082E20895E0E0F4E8EC0FFD1FA491DD
:101D2400BB2708957A2F0E945E3F803009F08FE030
:101D34000895AB2FBB270895CA2FAA27BB27C0300D
:101D440019F4A091220143C0C13029F4A0912201C9
:101D5400A030E1F33CC0C23039F4A0912201A0309C
:101D6400E1F7A091230133C0C33019F4A0912001FD
:101D74002EC0C43039F4C0912001C0FD1196C2FDBB
:101D8400119725C0C53039F4C0912001C1FD1196C9
:101D9400C3FD11971CC0C63049F4C0912201C23E54
:101DA40009F41197C33E99F4119611C0C73049F450
:101DB400C0912201C43E09F41196C53E41F4119725
:101DC40006C0D0912201CD17E1F7AC2FBB270895AF
:101DD400BB27A13021F4A0916D01A3950895A230F1
:101DE40021F4A0916E01A3950895A0916F01089527
:101DF4006F927F924F930E94D83F4030A9F0342FC6
:101E04003395ED010E94AA1C803071F521963E01A4
:101E14001A2F0027A02F0E9455420E942740141712
:101E240021F003950317B1F71CC0E3010E94AA1C1B
:101E34008030D1F4A03091F02A2FA02F0E94F442D8
:101E4400E3012196E8E8F1E00E94AA1C803061F4E5
:101E5400B191AB1731F721962A95B1F7A02FBB2783
:101E640002C0AFEFBFEF88274F917F906F90089526
:101E7400AA0FAA0FBA2FAA27C0E0D6E0CB27CC0F0F
:101E8400AA1FCB2FBB0FDA95C9F7AA0FAA0FBB273E
:101E94000895AA95A53048F40A2EA0E3BDE0A00D4C
:101EA400A00D0D901D90D0010895AA27BB27089579
:101EB400C8E7D1E008811981AA81BB818FDDB7FB16
:101EC40075DD2D010C811D81AE81BF8187DD82010D
:101ED4009EDD0C811D81A885B985F9017FDD66DD54
:101EE4002D0156944794E40DF51D421D521D422CBC
:101EF400522C320100E2EE0FFF1F441F551F441CF9
:101F0400551C661C771C4A165B066204720428F092
:101F14004A1A5B0A62087208E3950A9561F7DF01C1
:101F24000EF446CD088119815ACDFCE0E0EAA0E028
:101F3400B4EBA193BA95E9F7F1E0E8E6B0E1A19337
:101F4400BA95E9F7FDE0ECE3B0E0A193A193A19386
:101F5400BA95D9F7DD24CC2420921B0120921901D3
:101F6400AEE0A0933801ACE3A0935001AEE2A0939D
:101F74005101AFEFA0937701A093100120921301B8
:101F84000E94B93320925C01AFEFA0935201A09359
:101F94005301A2E0A0933F01A6ECA0937A004091E4
:101FA400490140934601409343010E9414799C2DBA
:101FB4000E941E7921D0803039F4AC2DAF35B8F3AE
:101FC4009CE020925C010895C0926D01D0926E0154
:101FD40080936F01813051F020925C014091770130
:101FE4004F3520F4DD24C42E8827E1CF9CE02092D5
:101FF4005C010895F7012AC0F1E0E0EB209236017C
:102004008827AD2DBB27AB1709F171917F3FD1F024
:102014007C31D1F07E31C1F07D31A9F07F3199F06E
:10202400773281F0723241F471917F3F59F0773207
:1020340049F07232C9F7E9CF7A3339F7B395AB1760
:1020440021F704C032C071917191DFCF70913901D1
:1020540070FD03C0803031F015C081E07E7F709345
:102064003901089572FF11C0AB7F70933901A091BB
:102074004A01A53011F0A03011F40E94E31FA0FF23
:1020840004C081E00F900F9008950E94BD387091B4
:102094001301703039F0A0911001DA9420921301E9
:1020A4000C94021471917F3F19F4DD24C3940895B4
:1020B40077FD2BC0703251F27A3311F4D394C6CF2A
:1020C400773201F27134D8F07B3528F070527134D4
:1020D400B0F07B35A0F4672E0E944F197D3379F45C
:1020E400C0DA803069F4762D7154770FDCE0C0EAF1
:1020F400C70FD21DA993B9937ECFEF91FF9187E0CB
:102104000895703810F487E075CF7F01EFE8F72F5A
:10211400FF73EF0FF0E1F21D09944EC0F7C0B7C290
:102124003DC112C1F8C230C391C73DC341C348C3C6
:102134003AC0D8C6F6C659C3CAC3DDC24FC47CC4AC
:1021440084C1C3C4D6C4DEC4F1C1ACC2E6C4F4C401
:10215400FBC4B5C556C1E2C091C235C150C5FEC469
:1021640029C053C56BC54CC2EBC218C621C06DC68D
:10217400D0C3DBC37FC1F4C647C7CCC773C682C60E
:1021840058C279C5A4C62BC1A4C2EBC304C3F4C40A
:10219400FAC449C181C186C6A1C188E0089584E119
:1021A400089583E1089576FD0C94081B0C94CC19D2
:1021B4000C94B4180C94E6190E9453199CE0732CE7
:1021C40020923601B191B032E9F3BA3321F0B7323B
:1021D40011F0BF3F59F4319770FC0E94FC334091D9
:1021E4003601453010F00E940A3F05CFBB3311F48D
:1021F4007724E8CFBC3291F440913601403031F479
:102204000E943434BA2DB770D9F706C00E94343412
:10221400B0913701B770D1F77724D4CF732CB33290
:10222400B9F420927801209279011BDA4A2F409365
:102234003601453008F4C6CF0E940E3F683059F588
:10224400509136015E7F0E94103F683121F5BACF6C
:10225400B03419F50E941A1940913601433018F42C
:102264000E94E835AFCF39F4A0937801B093790197
:10227400A0933701A7CF5FEF0E94103F683259F453
:102284005A2F0E94103F683231F45B2F0E94103F96
:10229400683209F497CF8FE00895B13229F4E1D977
:1022A4009A2F90CF98CF8ECFB23241F441914F3FC5
:1022B400C9F34232C1F30E943534F8CFB63291F4F7
:1022C400D0D9B33010F082E10895CCE3DDE0CA0F39
:1022D400DB1F4991403029F00E9435341196B33008
:1022E400C0F370CFB53229F4BCD94A2F0E943534DB
:1022F40069CF3197B6D9803009F00895903818F431
:102304000E9449335FCF0E94A4335CCF76FD0C94C6
:10231400EF1AA0E03FD70E94B9336CCEA2E03AD7BF
:10232400A03089F0B0917801BF70A13041F0A09144
:102334007A01A295A07FAB2B0E94F4325BCEAB2F27
:102344000E94193357CE2DCF76FD0C94AF1AA3E01B
:1023540021D7A33008F1A0917801B0917901A0931D
:102364007201B0937301A0917A01B0917B01A093A3
:102374007801B093790100917C0110917D011215CF
:10238400020549F00E94AE1C0E94BA1C803029F458
:1023940003191209F4CF2ECE04CF089576FD2ACE68
:1023A400A5E0F8D6A43070F00E94AB197F932FD724
:1023B400E0936B01F0936C010E9459377F91709305
:1023C400380118CEEECE76FD33C2A1E0E3D6A130BB
:1023D400C8F3409178014170409319010BCEA5E0F8
:1023E400D9D6A43068F0B5D77F9311D7E0936B01A9
:1023F400F0936C010E9472377F9170933801FACD8B
:10240400D0CEA5E0C7D6A43068F0A3D77F93FFD67B
:10241400C0936B01D0936C010E944C3C7F917093EC
:102424003801E8CDBECEA5E0B5D6A43068F091D78A
:102434007F93EDD6C0936B01D0936C010E94813CD5
:102444007F9170933801D6CDACCEA3E0A3D6A23051
:1024540080F07FD77F93B0917801A0917A01A09307
:102464006B01B0936C010E94FD357F91709338012C
:10247400C1CD97CEA5E08ED6A43068F06AD77F93FD
:10248400C6D6E0936B01F0936C010E94D4377F9120
:1024940070933801AFCD85CE76FD0C94711CA0915C
:1024A4004A01A03011F08CE10895A1E073D6A13067
:1024B40090F3A0917801B0917901CCE3DDE0CA0FEB
:1024C400DB1F409138014F93AF92BF920E94B63CFC
:1024D400BF90AF904F91409338018CCDA0914A01A9
:1024E400A03011F08CE10895BDD6D7D67C32E1F44A
:1024F400A1E051D6A13078F2A0917801B091790190
:10250400CCE3DDE0CA0FDB1F409138014F93AF925B
:10251400BF920E94F33CBF90AF90D2D249932992CC
:102524004F914093380166CD87E064CDA0914A0174
:10253400A03011F08CE1089595D6AFD67C32A1F786
:10254400A1E029D6A13009F02CCEFF93EF93AF92EE
:10255400BF92409138014F937F934F70409338015D
:102564000E949E1EC1E0D2E0ECE1F5E10E94B13789
:10257400C0913801C295C09338010E94CF3503023F
:102584000000A0917801B0917901CCE3DDE0CA0F9D
:10259400DB1FA6E14991403230F0403820F40E941C
:1025A4003534AA95B9F7772761E01FD00E94C01E81
:1025B400623061F485D2799329927F914F9140934F
:1025C4003801BF90AF90EF91FF9114CD7F914F915F
:1025D40040933801BF90AF90EF91FF9171D24FEFCC
:1025E4004993499307CD87E005CD0E94BE198827FA
:1025F400603009F408950E941D23882762E008953D
:10260400A3E0C8D5A230A0F0A4D67F93D0916C01EA
:10261400C0916B01F0917801E0917A01E0936B0134
:10262400F0936C010E94D4377F9170933801E2CC0F
:10263400B8CD76FD0C94811CA4E0ACD5A430C1F7D0
:10264400E6D5E8940E941237D5CCA4E0A3D5A430F3
:1026540079F7DDD568940E941237CCCCA4E09AD5E2
:10266400A43031F7D4D50E948537C4CCA4E092D5E8
:10267400A430F1F6CCD50E94B137BCCCA1E08AD508
:10268400A13078F0A09178010E942533B3CCA1E069
:1026940081D5A13030F0A0917801A150CA2EDD245B
:1026A40008957FCD76FD0BC0A1E074D5A13030F044
:1026B400A0917801A150A09377019CCC72CDA1E0A8
:1026C40069D5A130D8F3B091780168940E94AB3AEF
:1026D40091CCA7E05FD5A23088F3C8E7D1E0B881F8
:1026E400EA2FEA952296A8810E940933B395EA95C8
:1026F400C9F780CC56CDA1E04DD5A130D8F3A09137
:102704007801A7700E947C32A0914A01A73010F48E
:102714000E94B9336FCC76FD0C947C1BA1E03AD5B2
:10272400A13068F0A0917801B0917901B03019F42A
:10273400A03009F45FCC0E94FC371197F7CF31CD5C
:1027440020923F01A4E026D5A430C8F3CCE3DDE019
:10275400FE01A0917801B0917901B33098F4CA0FC9
:10276400DB1F00917A01A00FB21DA00FB21DB33080
:1027740048F4EA0FFB1FA0917C01B0917E010E94F6
:10278400E03E38CC82E136CC76FDCAC620925C01AC
:10279400BF91BF91089576FD0C946E1B84D5AB2B2D
:1027A40009F450CC28CC76FD0C94CF1A7AD523CCDE
:1027B40076FD0C94281BF7013BD50E94E8351BCC11
:1027C400A2E0E8D4A13080F029F4009053010092F3
:1027D400520105C0B0917A01E8940E94AB3AA091ED
:1027E40078010E94043807CCDCCCA6E0D3D4A13015
:1027F400D8F3B1E0EAE7F1E05BD0A0917801AA95C3
:10280400AF3510F08AE0F6CBB0917001B93010F01A
:102814008DE0F0CBAF93D3D0B064B993BC2DB99312
:10282400B0914901B993DD24CF9008950C94F31B22
:10283400A7E0B0D4A230C0F27232C1F3B2E0ECE748
:10284400F1E036D0409178014A950E9497794E3450
:1028540061F4F695E795A0917A015F3F11F0EA0FD4
:10286400F21D7096E8940995C5CBA0917A01AA95BA
:10287400AF35B8F7B0917801BA95B770B09343010A
:10288400B0917001B93010F08DE0B4CBAF9397D014
:10289400B064B993BC2DB993B0914601B993DD24CA
:1028A400CF9040914301409346010E9414790895CA
:1028B400C0E3DDE04A2F4B1B40933A0D403009F44E
:1028C400089551915993519159934A95F7CFA1E0A5
:1028D40061D4B0917001B03011F48CE00895A1304E
:1028E40041F4A0917801A0932E0DA0917901A093B9
:1028F4002F0DBA956CD0B0937001B991B6FFEDCF9E
:10290400BF70DB2EC9904991409346010E9414790F
:102914000895B0917001B93010F08DE06BCB4FD0B9
:10292400B062B993BC2DB99365CBB0917001BA95DF
:10293400A0F04DD0B991B5FF10C0B5D4AB2BB09178
:10294400700121F4BA95B093700155CBBA953FD07C
:10295400A991C990AF70DA2E08958EE0089587E0AA
:1029640008959FD49AD47134D0F37B35C0F7715451
:10297400770F672E92D47D3391F70E94330B80300A
:1029840009F00895DCE0C0EAC60DD21DA993B993FD
:1029940084D4733C21F70E94330B2D01803009F05D
:1029A4000895B0917001B93010F08DE0089507D00A
:1029B400B068B993C9926992499259921CCB07D0D5
:1029C400B395B0937001BD2DB395BF700895CCEF4E
:1029D400DCE0A5E0AB9FC00DD11D0895703C10F064
:1029E4000C9427135ED4B0917001B03011F48BE0D5
:1029F4000895BA95ECDFB991B7FFF9CFBF700B2EEC
:102A040059907991BCE0A0EAA70FB21D0D911D91D8
:102A1400030D121D1E930E93A991B99111960A17D5
:102A240041F41B1731F4B0917001BA95B093700161
:102A3400E2CAC52CD02C0895A0914A01A03011F00F
:102A44008CE108952ED4BFEFB0938801B191B032D8
:102A5400E9F34B2FBF3F21F40E94FC333197CBCADB
:102A6400BA33D1F3BB3391F3BC3231F40E94343422
:102A7400BA2DB770D9F7EACFB23241F441914F3F42
:102A840059F3423219F30E943534F8CFB134B0F01F
:102A9400BB35A0F4B154BB0FB0936A01B081B1341B
:102AA40018F0BB3508F40AC001D4DCE0C0EA109188
:102AB4006A01C10FD21DA993B993C8CF87E00895C5
:102AC400C0917201D0917301089576FD0C94301376
:102AD400EAD3803009F08FCA4A2F4B2BE1F340919F
:102AE4002E014030E1F340912E014030E1F711977F
:102AF400F3CF76FD0C943813D6D3A0932F01B09363
:102B04003001EACF76FD0C94961BACD3A0912F0133
:102B1400A993A0913001A9936ECA76FD0C94AD1BC4
:102B2400C2D34A2F0E946C39B9D37C3221F4B5D375
:102B34000E94330BF6CF5FCA76FD0C94CF1B0E9424
:102B4400C039A42FBB27C0C6F7017FD34A2FD73083
:102B540020F4C03D10F40E94893F4DCAF70175D39B
:102B64005A2FDE017091650177700E94533F0E94D5
:102B7400FC370E94FC373FCA76FD0C94471C93D364
:102B84006BD6A1B938CA76FD0C945A1CF7015DD3F3
:102B9400D030B9F461D6BC2FB770B39577276FE7FF
:102BA400A0FD70E8A0FD6FEF77FB770F70F967FB6E
:102BB400660F60F9BA95C1F702B1072B062302B973
:102BC4001ACAD13049F448D6B2B1C095BC23C095D5
:102BD400CA23BC2BB2B90FCAD23019F40E94921C7A
:102BE4000ACAD43019F4DD27A88305CAD83098F36B
:102BF4003BD640FF88E240FD0E940F72FCC976FD7F
:102C040017CE51D30E944A39F6C92CD30991199190
:102C1400105843D37C3281F418D3B058D058C0171D
:102C2400D10708F08E01A017B10708F48D0148DF21
:102C3400105809931993DFC986E00895A0914A01B9
:102C4400A63029F0A370A03011F08CE108950AD3C6
:102C54003E0123D37C3281F7EBD2C8EDD1E07EE193
:102C64007B9FC00DD11DCA0FD21DA881BB27E301D4
:102C7400A993B993C0C9A0914A01A370A03011F0DF
:102C84008CE10895EFD23E0108D37C32A9F6D0D26C
:102C9400C8EDD1E07EE17B9FC00DD11DCA0FD21DCE
:102CA400A2EBCA0FA2E0DA0FBB27A881A695BA2F20
:102CB400A777B295B078AB2BD9CF86E00895D2D25E
:102CC4003E01EBD27C32C9F7B3D2C8EDD1E07091AA
:102CD4004A0177707030E9F4AF93BF93A695B69527
:102CE4007EE17B9FC00DD11DCA0FD21D7881BF919B
:102CF400AF91A0FD7695B0FD7695B0FD7695A2EBEB
:102D0400B2E0CA0FDB1FA88170FFA295A695AF7031
:102D1400ADCF7130B9F4AF93A695A695A69575E19C
:102D24007B9FC00DD11DCA0FD21D7881AF91A2FD2A
:102D34007295A1FD7695A1FD7695A0FD76957170AD
:102D4400A72FE5CF7230A1F4AF93A695A6957EE1A7
:102D54007B9FC00DD11DCA0FD21D7881AF91A1FDFB
:102D64007295A0FD7695A0FF76957370A72FCFCFAF
:102D7400733071F4AF93A6957AE27B9FC00DD11D99
:102D8400CA0FD21D7881AF91A0FF7295A72FBFCF34
:102D9400AF93A695A695A69570E1C2CFA0914A01DE
:102DA400A63029F0A370A03011F08CE10895A3E0BF
:102DB400F1D1A33080F0A0917801B0917901B330C2
:102DC40010F082E10895B23039F4A73F28F082E18F
:102DD400089581E20895E5C9CCE3DDE0CA0FDB1F65
:102DE400C0936601D0935501AC81A03091F3AE310C
:102DF40080F7BB81B03069F3B73158F7C0917801DF
:102E0400D09179012596BA9F000C111C000C111C5D
:102E1400C00DC11DD330E8F6D0917A01C0917C0178
:102E2400C0935401D0935701CF3F51F0DF3F41F09D
:102E3400CA0FCA95CE3138F4DB0FDA95D73118F4BE
:102E44000E94623DD7C886E10895A0914A01A0304E
:102E540011F08CE1089525D2A0913901A460A093CA
:102E64003901C9C8A3E096D1A33009F09AC90E94D8
:102E7400A725403310F08EE108950E94BB258030D1
:102E8400D9F7B8C8A3E086D1A33009F08AC90E9453
:102E9400A725403310F08EE108950E94BE258030AE
:102EA400D9F7A8C8A3E076D1A23019F0A33021F055
:102EB40078C9A4E1A0937C010E94B525803009F46F
:102EC40099C808950E94B825803059F493C8A1E0A8
:102ED40061D1A13009F065C90E94A725443191F35D
:102EE4008EE10895A2E056D1A23009F05AC9A0910A
:102EF4007801B091790140917A01CCE3DDE0403072
:102F040041F0D395413029F0D395423011F082E15C
:102F140008950E94F33F0E94EF40803009F0089525
:102F240069C8A2E037D1A23009F03BC9A091780169
:102F3400B091790140917A01CCE3DDE0403041F079
:102F4400D395413029F0D395423011F082E10895B0
:102F54000E94B9400E940F40803011F3089550C080
:102F6400F7014AD1A09374010E940E3F6830B9F76B
:102F740090FF29C0592F0E94103F603481F7A03080
:102F8400D1F0DDE0CCE3409174014B0F4A1BC40F38
:102F9400D21DA13039F00E94143F603589F5588361
:102FA400AA95EFCF0E94193F683551F558830E94C6
:102FB4000A3F0C94FD0F0E94143F503099F3509334
:102FC4007401A52FDECF592F0E94103F6831C1F440
:102FD4003A2FDDE0CCE3409174014B0F4A1BC40F40
:102FE400D21D5881503011F4303031F00E94103F1E
:102FF400683231F4AA9569F70E940A3F0C94FD0FD8
:103004008FE00E940A3F08954ED1A0937801B093B7
:10301400790144D17C3249F431963FD1723239F08E
:1030240031970E94330BA4D4F4CF0C94FD0F71910B
:10303400723231F07F3F21F0BB27A72F99D4F7CF0D
:103044007081E7CFA43091F40C941A1AA7E0A2D0AF
:10305400B0917801B0935801B13051F0B03031F0F3
:10306400B23019F1B330F9F1B73060F385E1089566
:10307400A730E1F7C8E7D1E0BA81B0935501BC812C
:10308400B0936601BE81B0935601B885B0936701D1
:10309400BA85B0935701BC85B09354010E94F03AAD
:1030A400803009F008950C94FC0FA630F9F6C8E7B7
:1030B400D1E0BA81B0935501BC81B0936601BE8161
:1030C400B0935601B885B0936701BA85B0935401A3
:1030D400BB85B09357010E94F03A803009F00895FF
:1030E4000C94FC0FC3CFA430E9F7C8E7D1E0BA8150
:1030F400B0936601BB81B0935501BC81B093570175
:10310400BE81B09354010E94F03A803009F00895D2
:103114000C94FC0FA0914A01A03011F08CE10895A9
:10312400F70193D0C0937801D09379015091740141
:10313400A51708F45A2FA8E8B1E0503071F04D916A
:10314400A0937501B0937601A42FBB2711D4A0914D
:103154007501B09176015A95F0CFAA27BB2708D400
:103164000C94FD0FA0914A01A03031F0A43021F05D
:10317400A63011F08CE10895A1E00CD0A13040F00C
:10318400A09178014A2F43700E94243E0C94FC0FB6
:103194000C94D310F701A03009F40895DF93CF9372
:1031A400C8E7D1E040E05A2F503029F4A42F7F0122
:1031B400CF91DF910895DF93CF934F935F930E9454
:1031C400330B5F914F91CF91DF91893121F488279F
:1031D4007F01A42F0895A993B99343955A9550302C
:1031E40019F371917032E9F37C3229F33197A42FEA
:1031F4007F01CF91DF910895A3E0CCDFA33009F5DF
:1032040090917801B0917A01A0917C010895D091B8
:103214007801C0917A01F0917C01E0917E01C09324
:103224006601D0935501E0936701F0935601089528
:10323400A2E0B1DFA23029F4B0917801A0917A0123
:103244000895AF91AF910C94D310A2E0A4DFA23003
:10325400C1F7C0917801D0917901A0917A01B09120
:103264007B010895F70119D0713498F07B3558F437
:103274007154770FDCE0C0EAC70FD21DC09372010E
:10328400D09373010895713620F07B3710F4715692
:10329400F0CF8F918F9187E0089571917032E9F3A7
:1032A4000895F7010895F7010C94330BEF93FF93FE
:1032B4000E948A38FE0100E00E942F387091390183
:1032C400713011F4872F09C04A3EE9F40093740168
:1032D400003031F4AA27BB278827FF91EF91089586
:1032E400C8E8D1E0A191A9930A95E1F7AFEFA993BA
:1032F4000E94E61CE0EBF1E00E94330B8D010E947A
:103304001E79D801E9CF4C3E49F40030A9F2AA94C1
:103314000E948A38A0E2A8830A95CECF403230F2C8
:103324004B3720F6AA2DAD3108F60E9435340395AB
:10333400C3CF92E0BB27AC2DA3950E9449334AE347
:103344000E943534BB27AD2D0E9449330E9434348A
:10335400089570913801A0FF0895A33029F4A09135
:103364007C010E9419330895A53019F4A0918001BD
:10337400F8CFA0918401F5CF0E94C125403011F40B
:1033840066270895409380010E94B225413009F0D8
:1033940066270895A2E0FEDEA130A0F0B1E0A130DE
:1033A40011F0B0917A01A0917801A150A09310017D
:1033B400B09311010E94FC37B093120120921301C3
:1033C4000C94FC0F0C94D310A3E0E4DEC0917801BC
:1033D400D091790140917A0108EC1AE028ED31E0AE
:1033E400A23080F319F41CD00C94FC0F60917C0182
:1033F400F0917B01F170E0917A014CE3E40F4DE030
:10340400F41F4427C40FD21D41910AD04191403882
:10341400C8F34058C40FD21D6A9551F70C94FC0FA1
:10342400C017D10720F4DE01A20FB31F4C930895F7
:10343400FF93EF930CE310E120EA3CE0B0917801B4
:10344400B43019F5E8EDF1E0A0917A01B0917B0177
:10345400BF70AE0FBF1FC0917C01D0917D01DF70A2
:10346400CE0FDF1FE0917E01F0917F01A217B30719
:1034740040F4C217D30728F4319718F00D9009923D
:10348400F5CFEF91FF910C94FC0FB53009F5E8ED01
:10349400F1E0A0917A01B0917B01BF70AE0FBF1F24
:1034A400ECE3FDE0C0917C01D0917D01DF70CE0F93
:1034B400DF1FE0917E01F0917F01A217B30708F7A7
:1034C400C017D107F0F63197E0F20D900992F5CFCD
:1034D400B63011F5ECE3FDE0A0917A01B0917B01E7
:1034E400BF70AE0FBF1FE8EDF1E0C0917C01D09139
:1034F4007D01DF70CE0FDF1FE0917E01F0917F012F
:10350400A017B10740F4C217D30728F4319718F075
:103514000D900992F5CFB5CFEF91FF9185E1089514
:10352400A3E038DE70914A0150917A01409178010C
:1035340060917C01763021F0743041F00C94FC0FE2
:10354400A33051F40E94C93A0C94FC0FA23021F428
:103554000E94DD3A0C94FC0F35CFA2E01BDEA230B2
:1035640011F00C94D3100E94A725803009F008951F
:10357400403121F0483111F083E2089590917A01AD
:103584009A9570914601791731F0709178010E94F3
:103594008F240C94FC0F85E20895A2E0FBDDA23099
:1035A40011F00C94D3100E94A725803009F00895DF
:1035B4004C3F11F087E108957090490170917801B2
:1035C40090917A019A95909349010E94592470929E
:1035D4004901803001F00C94FC0FA2E0DBDDA23045
:1035E400D1F7A0E8B2E060917801C0917A01D0915E
:1035F4007C01CA17DB0740F4ACE3BDE0CA0FDB1F54
:103604000E94CD3E0C94FC0F82E10895A7E0C2DD38
:10361400A63038F19EDE7F9349D0C0936B01D093DE
:103624006C01E0917A01F09178010E94D43724D0A2
:10363400C0916B01D0916C01E0917A01F091780115
:103644000E94D4377F9170933801C5CFA7E0A2DDE3
:10365400A63038F07EDE7F9305D07F9170933801D9
:10366400BACFB0CEE8E6F1E021D0DE01E8E6F1E041
:10367400A383B4830E94FD35E8E6F1E0A08DB18D0B
:10368400C28DD38D2196AC17BD0708F0089511960D
:10369400A08FB18F0BD0E0916B01F0916C01C093BE
:1036A4006B01D0936C010E94D437E6CFA08DB18D0D
:1036B40034D0048911270E94FC0CD089DB1BA08D17
:1036C400B18D9D979D970E948F1B068911270E949B
:1036D400FC0CC289CB0F0895A1E05CDDA13030F071
:1036E400A0917801A0FF0E94BC3AA0FD0E94C43AB8
:1036F4000C94FC0FB7DDCF93DF93CFDDA5E04BDD5A
:10370400A53041F40E945A0FDF91CF91A993B99348
:103714000C94FC0FDF91CF91A4CFFF93EF930E9401
:10372400280DEF91FF9108959DDDB7DD7C3271F492
:10373400A1E031DDA13069F4A0917801B091790163
:103744006AD0BED9599329920C94FC0F87E00C944B
:10375400FC0F0C94D31086DDA0DD7C32B9F7A1E018
:103764001ADDA130B1F7E0917801F0917901E89484
:10377400F03818F0E095E3956894A2D9A881B9814E
:10378400E15038F01EF0AA0FBB1FFACFB695A795EB
:10379400F7CFA883B9830C94FC0F64DD7EDD7C3203
:1037A400A9F6A1E0F8DCA130A1F6E0917801F0914E
:1037B4007901E894F03818F0E095E395689480D99D
:1037C400A881B981E15048F01EF0AA0FBB1FFACFBF
:1037D4000B2E000CB795A795F5CFA883B9830C944D
:1037E400FC0F41914232A9F4EF014191423211F0B0
:1037F4004F3FD9F77F01409178014A950E9497790C
:10380400F695E79571964E3421F4689409950C94D5
:10381400FC0F0C94D310E0E0F0E93E9651E0659182
:103824006B1731F4A03019F065916A1709F4089503
:10383400F45FEE275395593091F750E008954F9374
:103844004A954770E6E0E49F4F91E8E0F8E4E00D24
:10385400F11DE50FF21D099407D041FF08950F9063
:103864000F9086E20C94FC0FEF93FF93EEE0F4EEDE
:10387400E4914427E03E30F0EF3F21F04160E03F27
:1038840008F04260FF91EF9108956091350164FD65
:1038940002C087E2089507DD4A2F0E947839FEDCD2
:1038A4007C3221F4FADC0E94330BF6CF0C94FD0F2A
:1038B40099276091350164FD03C087E20C94FC0FE5
:1038C4000E94D739A42FBB27409122014D3E11F409
:1038D400AFEFBFEFC7DCA993B9930C94FD0FA1E040
:1038E40059DCA130D8F0A09178016091350164FDD4
:1038F40002C087E208950E94A0390C94FD0FA1E054
:1039040049DCA13058F0A0917801A170B091180160
:10391400BE7FBA2BB09318010C94FD0F0C94D310F6
:10392400AF3F31F42C9A2CBCACE5ACBD2DBC089552
:10393400A7F92CBC2DBCA6FD3DBCAF73A064ACBDE7
:10394400A5B1A4FBA5B90895BDB5B7FFFDCF0895F2
:10395400AE01CF93DF9306C0CF93DF934091720102
:103964005091730110D0A991BB270EF4B99121C0D5
:10397400CF93DF93409178015091790104D0A993BA
:103984000EF4B99313C0DDE0CCE3533059F020F4C6
:10399400E894C40FD51F089568945450440F551FDC
:1039A4005330B8F34F914F9182E10895C8E7D1E0C5
:1039B40002C0C2E7D1E008801980030C121C0882FF
:1039C4001982DF91CF910895A0EBB1E04FEF52E25D
:1039D4004D935A95E9F7C8EAD1E040E25A91503242
:1039E40011F44A95D9F7442EA0EBB1E0C8E8D1E030
:1039F4004C0EA03D28F4C41518F44881403009F455
:103A040008958AD04F3FE1F371D04F3FC9F340305E
:103A140081F78FD0403069F73DD0403051F70AD05C
:103A2400403039F74991413618F04B3708F4405289
:103A34004D93DFCF4881403320F04A3310F4405394
:103A440002C044270895642F772721964881403384
:103A540080F04A3370F44053660F771F0B01660FF2
:103A6400771F660F771F600D711D640F721D2196FD
:103A7400EDCF703029F04DE14D937D936D93089512
:103A84006A3020F04CE14D936D930895605D6D9321
:103A94004CE108954881443211F044270895662783
:103AA4007727219658815033B0F05A3310F450538D
:103AB40008C05A3508F05052513468F0573458F45D
:103AC40057535F70529544E0550F661F771F4A9510
:103AD400D9F72196E7CF703029F04FE14D937D93CC
:103AE4006D9308954EE14D936D930895488142324C
:103AF40011F04427089521964D934991423219F4C7
:103B04004D9341E00895403029F442E24D934FEF44
:103B14004D9308954D93F1CF4881473211F04427D6
:103B2400089521964D9349914030E1F74FEF4D931D
:103B34000895FF93EF93BF93AF935F93E0E3F1E5B1
:103B44000E014591403089F0689457E0A591AE325A
:103B540039F0B991B13608F0B052AB1709F0E894D6
:103B64005A95A1F716F0E001EBCF5F91AF91BF91A9
:103B7400EF91FF91403041F04D934F934881403293
:103B840011F42196FBCF4F910895FF93EF93BF93C8
:103B9400AF935F930E014591403089F06894562F9E
:103BA400A591AE3239F0B991B13608F0B052AB17E5
:103BB40009F0E8945A95A1F716F0E001EBCF5F9174
:103BC400AF91BF91EF91FF91403049F04F934881FD
:103BD4004C3211F0403211F42196F9CF4F910895EF
:103BE400CBE8D1E0A0EBB1E040E2E0E24993EA9512
:103BF400E9F7A097A03D29F04D91423010F04F3FD6
:103C040011F429920895403220F0403810F486D0FF
:103C1400F1CF4C3121F4ED91FF2719D0EBCF4D3189
:103C240021F4FD91ED9113D0E5CF4E3131F444E20E
:103C340075D0ED91689449D0DDCF4F3131F444E231
:103C44006DD0FD91ED9134D0D5CF50D0D3CFE89441
:103C54004FE24395E051F742E0F7E05FF84D40331F
:103C640011F063D068944FE24395E85EF340E0F7C7
:103C7400E851FC4F16F0403311F057D068944FE2EE
:103C84004395E456F040E0F7EC59FF4F16F040330B
:103C940011F04BD068944FE24395EA50E8F7E65FA1
:103CA40016F0403309F041D040E34E0F3ED0089562
:103CB400E8944F2F42954F7011F012D068944F2F13
:103CC4004F700EF011F00CD068944E2F42954F7047
:103CD4000EF011F005D068944E2F4F7001D0089566
:103CE400405D4A3308F0495F20D00895E0E3F1E5F0
:103CF4005591503009F40895451711F03796F8CFCF
:103D04005F9357E045914E3209F00FD05A95D1F7A1
:103D14005F915C3110F040E208D008954993CB3AAA
:103D240018F029924F914F9108954993CB3AE0F3BB
:103D340029924F914F91F6CFA0914A01A0936E0121
:103D4400AA270E947C32A0913801A0936A01A09115
:103D54001B01A0936D01A0913601A09369012092EB
:103D64003601E8EDF1E0CCE3D7E0BEE2AEE141910B
:103D74004993AA95E1F7BA95C9F70895A0916E0100
:103D84000E947C32A0916D01A0931B01A0916A0155
:103D9400A0933801A0916901A0933601ECE3F7E008
:103DA400C8EDD1E0E2CFC6E1D4E0E8ECF6E041B101
:103DB40050B168E0A9E4BFEA469510F4AFE4BFE26D
:103DC400A993B193A0E3B0E8569510F4A1E3BEE43F
:103DD400AD8FB58F6A9571F70895452FA6E10E94BE
:103DE400F4324F5B0E9435344DE30E943534A7E131
:103DF4000E94F432C0EADCE0C50FD21DC50FD21D0B
:103E0400A991B9919DE00E9449330895A3E10E94CC
:103E1400E835A5E0C62FCA95AC9FCCEFDCE0C00D19
:103E2400D11DA881A6FF08C00E94CF35FF5355427B
:103E34002000A981AF7015C0A5FF06C00E94CF3530
:103E4400FF5250542000F5CF0E94CF35FF464F5209
:103E540020004A8146954F5B0E9435340E943434D9
:103E6400A981BB27A39592E00E9449334AE30E94AB
:103E74003534BB27A881AF700E944933089520923E
:103E84001B019927A7E00E94F4320E94B9330E94D3
:103E9400CF3512004249542030313233343536376D
:103EA40000000E94CF351300444952000E94CF35D0
:103EB40014004C455600E0E7F1E40E94393AA5E0CD
:103EC4000E94F4320E94CF3500004156522D4368BF
:103ED4006970426173696332204D4F4E2020202067
:103EE4005000409143014F5C0E9435340E94CF350D
:103EF400FF3A000092E0BB27AC2DA3950E94493302
:103F04000E94CF35FF3A0000BB27AD2DA3950E9438
:103F14004933EBE8F1E0C6EFD1E0AEE141EFB19116
:103F2400B03031F0BE8F4CAF4993AA95C1F706C0AB
:103F3400B0E2BE8F4CAF4993AA95D1F7A7E10E9496
:103F4400F432C0E0D4E0E1E1F0E1E8940E941237F9
:103F54009DE050E0452F4C5FB42FAA270E94E8351E
:103F64003CDF53955D30B1F7452F4950B42FA9E09C
:103F74000E94E83532DF53955A31B1F7A7E30E9426
:103F8400F432C3E1D4E0EDE1F0E1E8940E941237A9
:103F94000E94CF350413535441434B3A00009927F0
:103FA400BB27A09170010E9449336CE0C09170015D
:103FB400C61720F0C61BB4E0B60F28DF6A95B1F728
:103FC40008950E94B201AF92BF928F939F93B4DE83
:103FD40007DE55DF28D08827A09139014D3E11F422
:103FE400A16014C0413F11F4AA2710C0423F11F44C
:103FF400A4600CC0433F39F4C1DE0E942138AA27D3
:104004000E947C32E6CF443F29F716C0A0933901C1
:10401400409122014030E1F7B1DE9F918F91BF9032
:10402400AF900C94AD0120922301BDDE4091230199
:104034004030D9F30C94BD380E94283870E04424F1
:1040440025D0E2E5F1E40E94393A0E9421384D3E40
:1040540011F4A160DBCF443F19F40E942838B9CF92
:10406400463E31F4703069F37A950E942838E8CFDF
:10407400473E31F47A3028F773950E942838E0CF10
:10408400433FF9F643940E942838DACFA7E00E9410
:10409400F4320E94B9330E94CF350000417272613C
:1040A4007920566965772000A0E60E94F4320E94C8
:1040B400CF350200416472202000A0E50E94F43252
:1040C4000E94CF35020520202020202020202044DB
:1040D4006174612020202020202020202020000046
:1040E40060E4679FCCE3DDE0C00DD11DF00163E027
:1040F400A0E0B62F0E94E835A6E00E94F432DF016A
:1041040091E00E94A433A5E0B62F0E94E835A5E013
:104114000E94F43290E058E0A991B0E00E94A433E8
:10412400442D40FF0BC0A7E10E94F432219749912E
:104134000E943534A5E00E94F43202C00E94343457
:104144005A9551F738966395633191F60895204551
:104154007869742020202020202020202020202066
:10416400204368617220204D6F6E202020457869BD
:1041740074202020476F202020537465702020561F
:10418400696577202041727261792092360120920C
:104194004A01A5E00E94F432C0E0D0E0EDE1F6E18E
:1041A4000E94B137A0E50E94F4320E94CF3501028B
:1041B40044464C4153482073697A653A20000E9472
:1041C400C1254F3749F40E94CF35FF353132204B9A
:1041D40069427974650011C04F3F41F40E94CF35A4
:1041E400FF31204D69427974650007C00E94CF35C4
:1041F400FF3020427974650013C00E94B22541301B
:10420400D1F0EAE2F4E4E8940E94E639413009F49A
:1042140034C0453009F4B9CF423099F733D0B5CF23
:10422400E6E6F4E4E8940E94E639413009F425C056
:104234004530B1F7AACFEEEEF3E4E8940E94E639F4
:10424400413009F41AC0473019F40E9451229DCF1D
:104254004A3011F417D099CF423011F46DD095CF74
:10426400433019F40E94AA2290CF443019F40E94DA
:10427400FE228BCF4530F9F688CFA0912201A030E1
:10428400E1F708950E94EE3C4F466F726D61742011
:104294004D656469756D3F00413009F00895A6E2EB
:1042A4000E94F432C2E0D8E0EBE1FCE00E948537E2
:1042B4000E94CF350903466F726D617474696E672D
:1042C4002E2E2E202020202020000E94CF350B03EC
:1042D40000000E94C425803001F50E94CF350903F7
:1042E400466F726D617474696E672E2E2E20446F52
:1042F4006E652100A2E70E94F4320E94CF350B03C1
:10430400202020507265737320616E79206B65796B
:10431400212020000E94213808950E94CF350903EE
:10432400466F726D617474696E672E2E2E2045720D
:10433400726F72210000DECFA0E60E94F432C4E066
:10434400D8E0E9E1FDE00E9485370E94CF350905F8
:10435400417661696C61626C653A00000E94CF35F8
:104364000A0546696C65733A20009CE00E94A42506
:10437400DF93CF93DF010E9449330E94CF35FF20A2
:104384002F000E94C125A42FB0E011960E9449334A
:104394000E94CF350B05426C6F636B733A00AF918B
:1043A400BF910E9449330E94CF35FF202F000E9405
:1043B400AC25A0EFA49FD0011197B03009F4139756
:1043C4000E944933A6E00E94F4320E94CF350C05C6
:1043D400202020507265737320616E79206B65799B
:1043E400212020000E9421380895204578697420F6
:1043F40020496E666F204261636B757052657374F9
:104404006F7252657363616E202020202020446502
:104414006C6574652020202020202020202020206E
:10442400466F726D6174204578697420466F726DB1
:10443400617420202020202020202020202052656C
:104444007363616E20202020202020202020202043
:104454002020202020202020202020202020202058
:10446400202020457869742020202020202020202E
:104474002020202020202020202052657363616E9C
:104484002020202020202020202020202020202028
:1044940020202020202020202020202020207727BA
:1044A4000FD1A4E00E94F432C1E0D2E0ECE1F5E1E6
:1044B4000E94B137A0E40E94F4320E94CF35030277
:1044C40044656C6574652066696C6500B4D070934E
:1044D40078013BD34C3FD1F350D1413019F4A72F8D
:1044E400D5D244D308957727EBD0A4E00E94F432C8
:1044F400C1E0D2E0ECE1F5E10E94B137A0E40E9412
:10450400F432A0E1A0937C010E94CF3503025361F1
:10451400766520500000FFD28ED07093780115D3B9
:10452400403E30F4403171F0483161F0F6D0DCCFD8
:1045340009D3D03021F4CC3010F429D1D5CFA6D270
:10454400B6D108950ED1413079F6A0D2BCD10895E8
:104554007727B6D0A4E00E94F432C1E0D2E0ECE1C7
:10456400F5E10E94B137A0E40E94F432A2E1A093E5
:104574007C010E94CF3503024261636B75700000B9
:104584005AD070937801E1D2403920F4423161F07D
:10459400C4D0DFCFD7D2D03021F4C03610F4F7D056
:1045A400D8CF74D238D20895DCD0413091F66ED28F
:1045B4003ED20895772784D0A4E00E94F432C1E06B
:1045C400D2E0ECE1F5E10E94B137A0E40E94F432BC
:1045D4000E94CF3503024C6F6164205000009BD2CF
:1045E4002AD070937801B1D2403121F0483111F0D2
:1045F400A2D0E1CF90D10895772762D0A4E00E94A1
:10460400F432C1E0D2E0ECE1F6E10E94B137A0E47B
:104614000E94F4320E94CF350302526573746F72A4
:10462400650009D07093780190D2423111F08ED098
:10463400E4CF15D208957727B5D00BD10E94213845
:104644004D3E21F42FD14F914F9108954A3E09F4E4
:104654000895403E19F40FD17727EECF413E21F45F
:104664000AD170918001E8CF443E49F4703031F3AF
:1046740002D17150472F4F704F30F1F2DECF453EDB
:1046840059F440918001471709F4D8CFF4D07395B9
:10469400472F4F7089F2D1CF463E29F4703170F222
:1046A400EAD07051C9CF473E51F4409180014F3058
:1046B40031F04051471718F0DED0705FBDCFBECF48
:1046C4000E94C125403019F44F914F911BC0409373
:1046D40080010E94FC370E94FC3742D2413019F01D
:1046E4004F914F9101C008950E94B13C4F44464CF4
:1046F400415348206E6F7420666F726D61747465E7
:10470400640008950E94B13C4F44464C41534820F4
:104714006572726F7221000008950E94B13C4F438C
:10472400616E206E6F742073617665206F6E2074E5
:104734006869730008950E94B13C4F4E6F20424156
:104744005349432066696C65000008950E94B13C9A
:104754004F4E6F204241434B55502066696C6500B3
:1047640008950E94EE3CC04F766572777269746555
:104774002066696C653F000008950E94EE3C4F443A
:10478400656C6574652066696C653F0008950E94D8
:10479400B13C4F4E6F207370616365206C65667425
:1047A400000008955F936F937F93A72FA07FA0933A
:1047B4006C01A0916C01AF70AB5FBA2FA4E00E94B2
:1047C400E835A6E00E94F432A0916C01BB2795E085
:1047D4000E9449330E943434A5E00E94F432A0912F
:1047E4006C01A0937801B1D1B5D04F3F61F1A09194
:1047F4006C01A093780140E040937A0142E0409339
:104804007C018827B6D1803091F4CCE3DFE00E94AC
:1048140034345CE05F934991403808F04EE2403212
:1048240008F440E20E9435345F915A9599F7A091BB
:104834006C01A395A0936C01AF7009F0BACF7F917E
:104844006F915F9108955DE00E9434345A95E1F7C9
:10485400EECF4F935F93C4E2D5E0472F4F705EE1F4
:10486400459FC00DD11D52EF47E159934A95E9F791
:104874005F914F9108954F935F93C4E2D5E0472F22
:104884004F705EE1459FC00DD11D5CE044E059933B
:104894004A95E9F75AE043E159934A95E9F75F915C
:1048A4004F910895A0912201A030E1F708957093EB
:1048B40078014CE040937A0140E140937C0153D16C
:1048C400803009F01FCF7093780190914901ECE09A
:1048D400F0E99770929540EC949FE00DF11D0491DE
:1048E4003C9740E10E3409F448E10E94234040E043
:1048F4004F9300E0CCE3DFE0159119930A95E1F7BB
:1049040040937A0142E040937C0136D14F91439524
:104914004C3071F70895909149019770E0E0F0E907
:10492400929540EC949FE00DF11D40E04F9340932D
:104934007A0142E040937C01709378011AD1CCE370
:10494400DFE00E94587932964F9143954C3071F7CD
:1049540078940895403139F40E94CF35FF42415391
:104964003A0040E10895423139F40E94CF35FF42C4
:1049740055503A0042E10895443139F40E94CF354C
:10498400FF5553523A0044E10895463139F40E94E8
:10499400CF35FF4348383A0046E10895483139F4A9
:1049A4000E94CF35FF42494E3A0048E108954A310A
:1049B40039F40E94CF35FF47504F3A004AE1089539
:1049C4004C3139F40E94CF35FF53414D3A004CE14C
:1049D40008954E3139F40E94CF35FF4C424C3A00D1
:1049E4004EE108954F3139F40E94CF35FF494D47C8
:1049F4003A004EE10895403239F40E94CF35FF5316
:104A040043523A0040E208950E94CF35FF2D2D2DE8
:104A14002D004FEF08957093780140E640937A019A
:104A240042E140937C019FD0803009F06BCE7093BB
:104A340078014427E0E0F0E94F93CCE3DFE0002481
:104A4400159019920A94E1F740937A0142E0409359
:104A54007C0192D04F914395403671F7089540E020
:104A6400E0E0F0E94F9340937A0142E040937C0107
:104A7400709378017ED0CCE3DFE00E9458793296BF
:104A84004F914395403671F7789408950E94A2019E
:104A94004F9340913801409381014CE44093380195
:104AA400C6E0DAE0E7E1FCE00E9485370E94CF35FA
:104AB4000B0757726974696E6720646174612E2EE6
:104AC4002E0040918101409338014F910C949B0139
:104AD4000E94A2014F9340913801409381014CE41C
:104AE40040933801C5E0DAE0E8E1FCE00E94853754
:104AF4000E94CF350B0644617461207472616E7339
:104B04006665722E2E2E000040918101409338017B
:104B14004F910C949B01CCE3CCE340914901942F39
:104B24004F5C0E94353440E20E9435344091350197
:104B34004F934068409335010E948A794F91409386
:104B4400350108950E948F4108950E9453420E94A6
:104B5400274008950E94CA3F08950E945B4008952B
:104B64000E94714108950E94F84108950E945C4298
:104B740008950E94CC4208950E94724208950E94B2
:104B8400D83F08950E940E410895A1E00E944A3939
:104B94002092360120924A01A7E00E94F432C0E03C
:104BA400D0E0EDE1F6E10E94B137A0E70E94F432D3
:104BB4000E94CF35010243686970426173696332B0
:104BC40020636F6E6669677061676500A7E00E9485
:104BD400F4320E94CF351401436865636B73756DBD
:104BE4003A2000004FD100270E940B792091180130
:104BF400309165010E94283859D0EEECFEE4E89427
:104C04000E94393A0E9421384D3E09F40895423FEA
:104C140061F420931801309365010E9402790E9487
:104C2400FC370E94FC370C940000443E21F4013010
:104C340048F30A95DFCF453E21F4073018F7039572
:104C4400D9CF413FF9F6003031F4722F739571706A
:104C5400287F272BCFCF013029F44091180170E130
:104C64002727C8CF023019F478E02727C3CF0730AD
:104C740031F4732F3F78705F7077372BBBCF0330DD
:104C840031F4732F73957770387F372BB3CF04309B
:104C940021F4205C08F02064ADCF053011F43058C5
:104CA400A9CF063011F470E22727A4CFA6E00E9412
:104CB400F4320E94CF35030153657269616C20732D
:104CC400706565643A000E94CF350501493243207E
:104CD40073706565643A00000E94CF350701535034
:104CE400492073706565643A00000E94CF3509015C
:104CF400454550524F4D20616464726573733A00A8
:104D04000E94CF350B014C696E6520656E643A00D4
:104D14000E94CF350D0153657269616C20496E2F75
:104D24004F75743A00000E94CF350F0153657269C4
:104D3400616C20496E7075743A000E94CF35110180
:104D44004175746F73746172743A00001127B5D0A1
:104D540020FD09C00E94CF35031231323030204289
:104D64007073000008C00E94CF3503123234303013
:104D7400204270730000A1D024FD08C00E94CF35EA
:104D84000512313030206B487A0007C00E94CF35BD
:104D94000512343030206B487A008FD023FD08C0D0
:104DA4000E94CF35071235204D487A20200007C0D5
:104DB4000E94CF350712313536206B487A007DD0FA
:104DC4000E94CF3509120000432F4770405D0E94B6
:104DD400353473D0722F707C703841F40E94CF3513
:104DE4000B126F6E6C79204C460011C0703441F484
:104DF4000E94CF350B126F6E6C792043520007C0AE
:104E04000E94CF350B1243522B4C4620200055D024
:104E140037FD09C00E94CF350D1273696D706C6542
:104E24002020000008C00E94CF350D127374616EFB
:104E340064617264000041D025FF06C00E94CF3532
:104E44000F125044330005C00E94CF350F12504456
:104E5400310033D00E94CF35111250524720000048
:104E6400432F4295477039F0405D0E943534A7E0E6
:104E74000E94F43208950E94CF3511126F666620A5
:104E84002000F5CFAA27CC27DD27EE27FF27159092
:104E9400C10DD21DA21DFE38D1F7EE27F0EF1590FB
:104EA400C10DD21DA21DF030D1F7BB279FE00E9497
:104EB400A433DE010E94A4330895A5E0011709F488
:104EC400A0E50E94F4321395089520457869742072
:104ED4004368616E67652053617665202020202039
:104EE4002020202020202020AEE0A0933801C1E023
:104EF400D4E0ECE1F2E10E9485370E94CF3505054C
:104F040000000E94FB020E94CF35060320202020CF
:104F14002028632920323030362D323031302020A1
:104F24002020202000000E94CF35070320202020CD
:104F34006279204A6F65726720576F6C6672616D83
:104F4400202020200000A2EAA09338010E94CF353F
:104F5400090320202020202044656469636174656E
:104F64006420746F20202020202000000E94CF3570
:104F74000A03466C6F7269616E2C204572696B205E
:104F8400616E64204469616E612E0000AEE0A093FE
:104F940038010E94CF350C025468697320736F6620
:104FA4007477617265206973206C6963656E7365DB
:104FB40064000E94CF350D04756E646572207468B8
:104FC40065207465726D73206F66207468652000B7
:104FD4000E94CF350E04474E55205055424C49434C
:104FE400204C4943454E534520562E3320000E9401
:104FF400CF350F0355736520697420617420796F70
:105004007572206F776E207269736B210000A2ECB9
:10501400A09338010E94CF351107205052455353B5
:1050240020414E59204B455920000E9421380895B3
:105034009091490161E00E94C039509122015D3E86
:1050440009F408954531B1F7E0E0F0E997709295DD
:1050540040EC949FE00DF11DCCE3DDE050E0459180
:1050640049935A95E1F7CCE3DDE00E94CD3E0E94DE
:10507400C039509122015D3E21F34630A1F763957A
:10508400CCEBDDE00E94CD3E0E94C039509122015C
:105094005D3EB9F24630A1F763956931E9F644E023
:1050A4000E946C390895909149019770E0E0F0E90D
:1050B400929540EC949FE00DF11D45E10E946C39FE
:1050C40060E06F93CCE3DFE00E94AA3E803041F0C1
:1050D400813051F1843241F145E10E946C39F2CFC3
:1050E40046E00E946C39CCEBDFE00E94AA3E80309F
:1050F40041F08130C9F08432B9F045E10E946C3945
:10510400F2CF0E9458797894329646E00E946C3926
:105114006F9163956C30A9F60E9485394430E1F7AC
:1051240046E00E946C3908956F91089502414253FC
:10513400282E2E2E0353474E282E2E2E0453515222
:10514400282E2E2E054E4F54282E2E2E06524E4417
:10515400282E2E2E07414443282E2E2E08494E2851
:105164002E2E2E2E09585045454B282E0A54454DB7
:1051740050282E2E0B4C4F282E2E2E2E0C4849280C
:105184002E2E2E2E0D4B4559282E2E2E0E455045D3
:10519400454B282E0F455252282E2E2E10415228B0
:1051A4002E2E2E2E1153494E282E2E2E12434F539F
:1051B400282E2E2E134654595045282E1446534952
:1051C4005A45282E155053544154282E16535049ED
:1051D400282E2E2E174D454E55282E2E1856504546
:1051E400454B282E1958524543282E2E1A46464917
:1051F4004E44282E1B44424954282E2E8050524996
:105204004E542E2E81434C532E2E2E2E82474F5415
:105214004F2E2E2E83424F582E2E2E2E8441434F36
:1052240050592E2E8553594E432E2E2E86454E44CC
:105234002E2E2E2E8742434F50592E2E88544845E9
:105244004E2E2E2E89504F532E2E2E2E8A4E4F54D4
:10525400452E2E2E8B4F4E53594E432E8C52524573
:1052640041442E2E8D5257524954452E8E474F534A
:1052740055422E2E8F52455455524E2E90564D4F18
:1052840044452E2E914E4558542E2E2E92494E5062
:1052940055542E2E93504C4F542E2E2E9457414934
:1052A400542E2E2E95545345542E2E2E9654474547
:1052B400542E2E2E974653454C454354984F4E45F5
:1052C40052522E2E99535055542E2E2E9A534745F2
:1052D400542E2E2E9B45504F4B452E2E9C47455405
:1052E4005049582E9D434952434C452E9E434F4CA2
:1052F4004F522E2E9F424F524445522EA0464F4E9F
:10530400542E2E2EA150554D502E2E2EA258504FB5
:105314004B452E2EA356504F4B452E2EA44C494D93
:1053240049542E2EA547455443484152A644524160
:1053340057544F2EA7504C41592E2E2EA85350523D
:105344004954452EA95343524F4C4C2EAA42524520
:10535400414B2E2EAB5245504541542EAC554E5424
:10536400494C2E2EAD445241572E2E2EAE49434F5A
:105374004D4D2E2EAF444154412E2E2EB043544554
:1053840058542E2EB146524541442E2EB246575201
:105394004954452EB343424F582E2E2EB4474554FC
:1053A40041545452B54644454C455445B646424F83
:1053B400582E2E2EB750414C45545445B8464F52A2
:1053C4002E2E2E2EB949462E2E2E2E2EBA4449525A
:1053D4002E2E2E2EBB4F55542E2E2E2EBC46434918
:1053E40052434C45BD414C4552542E2EBE46435269
:1053F40045415445BF41534B2E2E2E2ECE474F537D
:105404002E2E2E2EC03F2E2E2E2E2E2EC15853451C
:105414004E442E2EC2474F2E2E2E2E2EC3544F2EC8
:105424002E2E2E2EC44C4F4144502E2EC553434194
:105434004C452E2EC643434841522E2EC742432E7E
:105444002E2E2E2EC853415645502E2EC94152435E
:105454002E2E2E2ECA4E4F2E2E2E2E2ECB5049459A
:105464002E2E2E2ECC5252442E2E2E2ECD5257524C
:105474002E2E2E2ECF5245542E2E2E2ED0564D2E5D
:105484002E2E2E2ED149424F582E2E2ED2494E501A
:105494002E2E2E2ED3504C2E2E2E2E2ED44652414E
:1054A4004D452E2ED5484652414D452ED64C4649A3
:1054B4004E442E2ED74653454C2E2E2ED8564F4CA6
:1054C4002E2E2E2ED94C53484946542EDA41534899
:1054D4004946542EDB45502E2E2E2E2EDC47505896
:1054E4002E2E2E2EDD43492E2E2E2E2EDE434F4CF5
:1054F4002E2E2E2EDF424F2E2E2E2E2EE043414CEA
:105504004C2E2E2EE143412E2E2E2E2EE258502EBE
:105514002E2E2E2EE356502E2E2E2E2EE44C494D9A
:105524002E2E2E2EE54743482E2E2E2EE644544F83
:105534002E2E2E2EE85350522E2E2E2EEB52455048
:105544002E2E2E2EEC554E542E2E2E2EED44522E53
:105554002E2E2E2EEE49432E2E2E2E2EEF44412E8D
:105564002E2E2E2EF14652442E2E2E2EF246575219
:105574002E2E2E2EF3424155442E2E2EF447415406
:105584002E2E2E2EF54644454C2E2E2EF750414CF1
:105594002E2E2E2EF95649442E2E2E2EFA455350D9
:1055A40055542E2EFB45534745542E2EFC46434955
:1055B4002E2E2E2EFD45424155442E2EFE4643529C
:1055C4002E2E2E2E002E2E2E2E2E2E2EA091140197
:1055D400B0911501ED01E2EBF2E0CE0FDF1FF6EF23
:1055E400E0911A01FE0F7F934F92EEE14E2E6991E6
:1055F400ED915491762F7295762757FD672768B9F8
:10560400ED91000056FD76B9049055FD76B9699187
:10561400162E54FD76B91294162653FD76B907FC5E
:1056240061254A9452FD76B9502D712D41F7609150
:105634001B0168B94F907F91EE91F0911A01F39597
:10564400FA3029F4FF27A0931401B0931501F093C5
:105654001A010C946E31A0911401B0911501F82D2A
:10566400FA95CCE5DBE0F295FF70E5E1EF9FC00D24
:10567400D11D10901B01FD916991462FF0FD4295BB
:1056840048B9562F452FF1FD429548B90000452FE2
:10569400F2FD429548B96991452FF3FD429548B909
:1056A4000000452FF4FD429548B90D90452FF5FDB6
:1056B400429548B90000452FF6FD429548B9F7FDDB
:1056C4005295462F00FC429558B9F02DEA95C1F643
:1056D40018B8EE91F0911A01F395F23029F4FF27EE
:1056E400A0931401B0931501F0931A010C946E3138
:1056F400A0911401B0911501D1E0FEE110901B01BD
:10570400ED91CE2FC370588158B9CE2FC695C6954A
:10571400C3705881E29558B9CE2FC3705881CE2FEB
:10572400C69558B9C695C3705881ED91CE2F58B916
:10573400C3705881FA9541F718B8EE91F0911A01A7
:10574400F395F33029F4FF27A0931401B0931501C6
:10575400F0931A010C946E31A0911401B0911501CB
:105764000F9310901B01EAE2D1E0CD9100000C2FC1
:105774000295CF70F881F8B9C02FCF70F88100007E
:1057840000000000F8B9CD9100000C2F0295CF70F5
:10579400F881EA9581F718B811970F91F0911A01E1
:1057A400F395F43029F4FF27A0931401B093150165
:1057B400F0931A010C946E31A0911401B09115016B
:1057C400D0910001C0910101C295DC0FDE7EE0E1C1
:1057D40010901B01FD914D2FF0FD429548B900003A
:1057E400000000004D2FF1FD429548B90000000073
:1057F40000004D2FF2FD429548B9000000004D2FE6
:10580400F3FD4295000048B9000000006D2F4D2FB4
:10581400F4FD429548B90000CD91F5FD62955D2FE8
:1058240068B900000000F6FD52956D2F4D2F58B950
:10583400F7FD6295C0FD42950000000068B9FC2F99
:1058440000000000EA9551F6000018B8EE91F091BE
:105854001A01F395F33029F4FF27A0931401B093B0
:105864001501F0931A010C946E31A0911401B091BA
:105874001501C0914D01D82DF6EFE0911A01FE0FEC
:10588400E395E0931A01EA3088F1EC3069F59396D8
:10589400A0931401B093150120921A01DC3031F465
:1058A400D0914C01D0934D010C946E31D83189F4D0
:1058B400A1E4B2E0C0913A01D3E2CD9FA00DB11DA5
:1058C400CEE0A0931401B0931501C0934D010C9444
:1058D4006E31D83D49F4CBE4AEE1B2E0A0931401BB
:1058E400B0931501C0934D010C946E310F931F9327
:1058F4002F93D83D28F4DC2F0C2F1C2F2C2F05C000
:1059040028E61CE208E8DCECCAE46C2F7C2F7295D4
:10591400ED91E7FD6727EF775491ED9168B9172E64
:1059240056FD16B86C2F7C2F729555FD16B8E7FD01
:10593400672754FD16B8EF77000053FD16B804909E
:1059440052FD16B8502DED9168B9172E56FD16B8B4
:105954006C2F7C2F729555FD16B8E7FD672754FD13
:1059640016B8EF77000053FD16B8049052FD16B830
:10597400502DED9168B9172E56FD16B86C2F7C2F5B
:10598400729555FD16B8E7FD672754FD16B8EF77F5
:10599400000053FD16B8049052FD16B8502DED9139
:1059A40068B9172E56FD16B86C2F7C2F729555FDCD
:1059B40016B8E7FD672754FD16B8EF77000053FDCE
:1059C40016B8049052FD16B8502DED9168B9172EF3
:1059D40056FD16B86C2F7C2F729555FD16B8E7FD51
:1059E400672754FD16B8EF77000053FD16B80490EE
:1059F40052FD16B8502DED9168B9172E56FD16B804
:105A04006C2F7C2F729555FD16B8E7FD672754FD62
:105A140016B8EF77000053FD16B8049052FD16B87F
:105A2400502DED9168B9172E56FD16B86D2F7D2FA8
:105A3400729555FD16B8E7FD672754FD16B8EF7744
:105A4400000053FD16B8049052FD16B8502DED9188
:105A540068B9172E56FD16B86D2F7D2F729555FD1A
:105A640016B8E7FD672754FD16B8EF77000053FD1D
:105A740016B8049052FD16B8502DED9168B9172E42
:105A840056FD16B86D2F7D2F729555FD16B8E7FD9E
:105A9400672754FD16B8EF77000053FD16B804903D
:105AA40052FD16B8502DED9168B9172E56FD16B853
:105AB4006D2F7D2F729555FD16B8E7FD672754FDB0
:105AC40016B8EF77000053FD16B8049052FD16B8CF
:105AD400502DED9168B9172E56FD16B86D2F7D2FF8
:105AE400729555FD16B8E7FD672754FD16B8EF7794
:105AF400000053FD16B8049052FD16B8502DED91D8
:105B040068B9172E56FD16B86D2F7D2F729555FD69
:105B140016B8E7FD672754FD16B8EF77000053FD6C
:105B240016B8049052FD16B8502DED9168B9172E91
:105B340056FD16B86D2F7D2F729555FD16B8E7FDED
:105B4400672754FD16B8EF77000053FD16B804908C
:105B540052FD16B8502DED9168B9172E56FD16B8A2
:105B6400602F702F729555FD16B8E7FD672754FD19
:105B740016B8EF77000053FD16B8049052FD16B81E
:105B8400502DED9168B9172E56FD16B8602F702F61
:105B9400729555FD16B8E7FD672754FD16B8EF77E3
:105BA400000053FD16B8049052FD16B8502DED9127
:105BB40068B9172E56FD16B8602F702F729555FDD3
:105BC40016B8E7FD672754FD16B8EF77000053FDBC
:105BD40016B8049052FD16B8502DED9168B9172EE1
:105BE40056FD16B8602F702F729555FD16B8E7FD57
:105BF400672754FD16B8EF77000053FD16B80490DC
:105C040052FD16B8502DED9168B9172E56FD16B8F1
:105C1400602F702F729555FD16B8E7FD672754FD68
:105C240016B8EF77000053FD16B8049052FD16B86D
:105C3400502DED9168B9172E56FD16B8602F702FB0
:105C4400729555FD16B8E7FD672754FD16B8EF7732
:105C5400000053FD16B8049052FD16B8502DED9176
:105C640068B9172E56FD16B8612F712F729555FD20
:105C740016B8E7FD672754FD16B8EF77000053FD0B
:105C840016B8049052FD16B8502DED9168B9172E30
:105C940056FD16B8612F712F729555FD16B8E7FDA4
:105CA400672754FD16B8EF77000053FD16B804902B
:105CB40052FD16B8502DED9168B9172E56FD16B841
:105CC400612F712F729555FD16B8E7FD672754FDB6
:105CD40016B8EF77000053FD16B8049052FD16B8BD
:105CE400502DED9168B9172E56FD16B8612F712FFE
:105CF400729555FD16B8E7FD672754FD16B8EF7782
:105D0400000053FD16B8049052FD16B8502DED91C5
:105D140068B9172E56FD16B8612F712F729555FD6F
:105D240016B8E7FD672754FD16B8EF77000053FD5A
:105D340016B8049052FD16B8502DED9168B9172E7F
:105D440056FD16B8612F712F729555FD16B8E7FDF3
:105D5400672754FD16B8EF77000053FD16B804907A
:105D640052FD16B8502DED9168B9172E56FD16B890
:105D7400612F712F729555FD16B8E7FD672754FD05
:105D840016B8EF77000053FD16B8049052FD16B80C
:105D9400502DED9168B9172E56FD16B8612F712F4D
:105DA400729555FD16B8E7FD672754FD16B8EF77D1
:105DB400000053FD16B8049052FD16B8502DED9115
:105DC40068B9172E56FD16B8622F722F729555FDBD
:105DD40016B8E7FD672754FD16B8EF77000053FDAA
:105DE40016B8049052FD16B8502DED9168B9172ECF
:105DF40056FD16B8622F722F729555FD16B8E7FD41
:105E0400672754FD16B8EF77000053FD16B80490C9
:105E140052FD16B8502DED9168B9172E56FD16B8DF
:105E2400622F722F729555FD16B8E7FD672754FD52
:105E340016B8EF77000053FD16B8049052FD16B85B
:105E4400502DED9168B9172E56FD16B8622F722F9A
:105E5400729555FD16B8E7FD672754FD16B8EF7720
:105E6400000053FD16B8049052FD16B8502DED9164
:105E740068B9172E56FD16B8622F722F729555FD0C
:105E840016B8E7FD672754FD16B8EF77000053FDF9
:105E940016B8049052FD16B8502DED9168B9172E1E
:105EA40056FD16B8622F722F729555FD16B8E7FD90
:105EB400672754FD16B8EF77000053FD16B8049019
:105EC40052FD16B8502DED9168B9172E56FD16B82F
:105ED400622F722F729555FD16B8E7FD672754FDA2
:105EE40016B8EF77000053FD16B8049052FD16B8AB
:105EF400502DED9168B9172E56FD16B8622F722FEA
:105F0400729555FD16B8E7FD672754FD16B8EF776F
:105F1400000053FD16B8049052FD16B8502DED91B3
:105F240028B82F911F910F910C946E31A0911401F8
:105F3400B0911501EAE8F4E0C0911A01D3E0CD9FD5
:105F4400E00DF11D7F936EE17EE1CBE1D1E058815C
:105F5400507F452F4295542B588358B952954D91F3
:105F64004F7358B95991469F58B95295EF010000A3
:105F740058B9C00DD11D599158B952957A95000060
:105F8400000058B9599149F7000058B952956091E9
:105F94001B01000058B959917F9158B95295F0915D
:105FA4001A01F39558B90000000068B9FA3029F4D1
:105FB400FF27A0931401B0931501F0931A010C94D8
:105FC4006E31A0911401B0911501ED01E2EBF2E004
:105FD400CE0FDF1FF7E0E0911A01E395E0FBE695B1
:105FE400FE0F7F934F92EEE14E2E6991ED91E7F90A
:105FF4005081762F7295762757FD672768B9ED9102
:10600400E7F956FD76B90080000055FD76B969912F
:10601400162E54FD76B91294162653FD76B907FC54
:1060240061254A9452FD76B9502D712D39F760914E
:106034001B0168B94F907F91EE91F0911A01F3958D
:10604400FA3029F4FF27A0931401B0931501F093BB
:106054001A010C946E3128B818954F935F936F937F
:10606400FF93EF93DF93CF93BF93AF930F921F925E
:10607400FFB7FF9330921D01B0913D01B7FF5C98CB
:10608400B7FD5C9AC0911801A0916501D9B1D3FB09
:10609400C5FFD1FBB0F9A7FFB325B0933D01C4E11F
:1060A400D1E05F89A889E9890A881B88A00DE11DD0
:1060B400A88BE98BFFA14491AD89AF73AF3309F489
:1060C400452F5AA5BEADB59F512D4503B0E8B10D7E
:1060D400B093B300EE89FF89488D598DA52FAA0F7F
:1060E400EE1FFF1F441F551F40F4ADE5EA27A5ED41
:1060F400FA27AAE24A27A5ED5A27EE8BFF8B488F91
:10610400598F830C921CEBA9FF81EF23E8B9789493
:10611400E9A190FC04C0F8A58F1608F4A7C071F497
:10612400409110014F3F51F0409112014A9521F4E2
:10613400409111013092130140931201FCE0E2FFFF
:10614400FDEE8F1639F45E98E3FFC6C0B2E8B09353
:106154008000C2C0F1E1E2FFF3EF8F1639F45E9ADA
:10616400E3FFBAC0B2ECB0938000B6C0FBE1E2FF3B
:10617400FFEF8F1621F4EFEFE0934701ADC0F2E09B
:10618400E2FFFCEE8F1619F420924701A5C0F9E353
:10619400E2FFF7E08F1609F09FC0A8EDA883A1E005
:1061A400A9832E8288249924AAE0A9AFA5E0E2FF5E
:1061B400A39542E3E2FF4CE3BA8DB395BA1731F4E9
:1061C400BB27EB8DFC8D3196EB8FFC8FBA8FE88566
:1061D400E395E41709F4EE27E887FDE8E0E0A091F1
:1061E4002901A7FDB096AC89EA0FF21DB491B2154E
:1061F40011F0A395AC8BBAA760913F016030A9F16F
:10620400B0915D01BA95B0935D0179F5B0915C01EF
:10621400B0935D01B0916401BA95B093640129F51E
:10622400E0915E01F0915F01C0916201D091630140
:106234002197A191B1914B2FB295BF7019F0E894B9
:106244000E94AB3A4F7040936401DCD6EC17FD0713
:1062540040F067FF6A9560933F01E0916001F0911F
:106264006101E0935E01F0935F0136C0A091840068
:10627400AB3EE0F3AC3E00F0AD3E00F0AE3E00F0CD
:10628400AF3E00F0E5FD28C0E0913501E7FD0C9438
:10629400372CE0914A01E53011F40C94DE2BE03008
:1062A40011F40C94E82AE13011F40C942D2BE23013
:1062B40011F40C947A2BE43011F40C94E32FE630AF
:1062C40011F40C94982FE73029F4C8EDD1E00E9422
:1062D400177202C00C94AE2BA0912001A5FD23C01F
:1062E400E091C000E7FF67C0E091C600E093710150
:1062F400F5EFB491B0FF32C0A7FF03C02092220192
:1063040057C0E33809F4E0E1F8E8EF77A4FFA6FD0D
:10631400F395A4FFA0FDE068A1FDE068E491E0939B
:106324002101A06246C0E0912101E0932201E093A3
:106334002301EE3E19F4A2FD0C9451014091390160
:10634400E33611F4A2FD4160E03711F4A3FD42608D
:10635400EC3F09F44460409339012AC0E03F11F452
:10636400A06827C0E03E11F4A06423C0E23131F4F8
:10637400A6FD1EC0A160A7FDAE7F1AC0E93521F4B9
:10638400A260A7FDAD7F14C0E43151F4A6FD04C0A2
:10639400A460A7FDAB7F0CC0A860A7FDA77F08C0C1
:1063A400E13121F4A061A7FDAF7E02C02092220159
:1063B400AF71A09320014091180140FD0E949C7888
:1063C40040FF0E94D178FF91FFBF1F900F90AF91C3
:1063D400BF91CF91DF91EF91FF916F915F914F91B9
:1063E4001895AAEBA4B9AFEFA5B9A0EFA7B9A0E09F
:1063F400A8B9A0EFAAB9AFEFABB9A6B1AE70A0939C
:106404003501B2ECB0938000B9E1B0938100F4E0BF
:10641400A2FFF4E0F0938700FEEFA2FFF6EFF09303
:10642400860020928900FAE5F0938800F4E0F09366
:106434008B00F8EDF0938A00A6E0A0936F00A2E031
:10644400A4BDA1E0A5BDA1E3A7BDA3E8A093B000AE
:10645400A1E0A093B100A0E8A093B3002092B600FD
:106464002092C000A0E1A093C100A6E6A093C200C0
:106474002092C9000E940B79B0911801B5FD09C0A2
:10648400A3E05CD7A8E1A093C900A6E0A093CA004A
:10649400539AACE5B3FDAFE5ACBDA0E0ADBDA5E15D
:1064A400A1D0C4E1D1E0A8EDA993A1E0A993AEE104
:1064B4002992AA95E9F7AAEAA0932A01A0932C01AC
:1064C4002092360120921901AEE3A09328010F9384
:1064D400009135010F770093350106EE07C00F9345
:1064E4000091350100680093350104EE00933C01EE
:1064F4000F9108950F01EEE0F4EEB491F001BF3F67
:1065040031F0B07EB03E19F4E8940E9411723A2F33
:10651400A03021F0A43051F40E94963AACE3A09349
:106524005001AEE2A0935101A6EE43C0A13069F43C
:10653400A8EAA0935001A4E7A0935101A0E0A0937E
:106544000001A0EEA093010123C0A23091F4A8E7BA
:10655400A0935001ACE4A0935101C0E0D1E0A0E0CD
:10656400A883A0E4A983A0EAAA83A0EEAB83A3EE48
:1065740020C0A33079F4A4E5A0935001AAE3A0932A
:106584005101AA27B0E043D0A395B395B031D9F710
:10659400A7EE0FC0A53091F4A0E8A0935001A0E4A9
:1065A400A0935101A0E2A0930001A0EEA0930201E8
:1065B400A0ECA0933C0130934A010895A63051F415
:1065C400ACE3A0935001AEE2A09351010E94633A60
:1065D400A6EEEFCFB03E11F085E0089568940E94D6
:1065E4001172E7CFBF93AF93BA2FB878B695B6952B
:1065F400B695AA0FAE7EAB2BA0933801AF91BF9195
:106604000895A09336010895A09319010895DF9386
:10661400CF93AF93AF70A295AA0F08F4A061D1E015
:10662400CB2FCF70A883AF91CF91DF910895BF9303
:10663400AF93AF70A295AA0F08F4A061A295B09190
:106644003801B07FD8CFAF93A295A7FBAA0FA4F9C6
:10665400A07FA0931B01AF91089548834091350119
:1066640047FD14C040914A01463081F0CF93DF9337
:106674005F935CE3C50FD21D46E7C40F42E0D41F0D
:106684004091380148835F91DF91CF9108954F93F2
:106694005F936F93AF93BF9340E2592F537052307F
:1066A40061F0533009F44BE2B7FF05C0A095B095F3
:1066B400A30DB21D4DE20E943534592F5C70692F31
:1066C4006073E8944FE24395A051B742E0F7A05FAE
:1066D400B84D5C3009F42BD04FE24395A85EB3402B
:1066E400E0F7A851BC4F53FD22D0603309F4B8D071
:1066F4004FE24395A456B209E0F7AC59BF4F50306E
:1067040009F015D0603209F4ABD04FE24395AA509A
:10671400E8F70DD0A65F603109F4A2D040E34A0F38
:10672400A2D0BF91AF916F915F914F910895403383
:1067340011F0689498C091FD96C0F6F390FF089507
:1067440091C008954F9390FF05C04B2F429509D0F7
:106754004B2F07D04A2F429504D04A2F02D04F9195
:1067640008954F70405D4A3308F0495F7CC00E9431
:10677400A20140914A01403009F14430F9F0D1E0DE
:10678400C8EDA7E1463019F0473061F1ACE5BEE150
:106794002992BA95E9F7AA95D1F7413069F4A09105
:1067A4003801DBE0CCE5B0EAA993A993BA95E1F707
:1067B400AA24BB24209237010C949B0140E2D1E02F
:1067C400C8EDA7E1BEE14993BA95E9F7AA95D1F7D7
:1067D40040913801A7E1BEE14993BA95E9F7AA953A
:1067E400D1F7E6CF0E941272E3CF20923701BF9116
:1067F400AF910895AF93BF9320923701A0913601D2
:10680400A03051F4A7E1AA24B394AB1571F7B6E113
:10681400BB2ECF93DF937CC0A13021F4BF91AF9105
:106824000C945239A23059F44DE0B0911801B6FDE0
:106834008AD44AE0B7FD87D4BF91AF910895A330BD
:1068440019F4BF91AF910895A43021F4BF91AF9191
:106854000C945F39BF91AF915AE00E94103F0895A4
:106864004CE201C040E2AF93BF93A0913701A395DE
:10687400A0933701A0913601A53030F0BF91AF91BC
:10688400542F0E94103F0895A030D1F0A33059F442
:10689400A42FBB275F936F930E94BA1C6F915F91E3
:1068A400BF91AF910895BF91AF91A0913601A130EE
:1068B40011F40C946C39A23009F445C40C94783961
:1068C400EF93E0914A01E03061F0E43051F0E630BA
:1068D40041F0E73029F4EF91BF91AF910C9413721A
:1068E40098C0EF91CF93DF9313D496FD33C0B5DEF8
:1068F400A395AE3131F4AA27B395B73111F4B6E1BB
:1069040006C05D01DF91CF91BF91AF9108955D0104
:10691400D1E0C8ED4F93A6E1BEE14E8D4993BA95FF
:10692400E1F7AA95C9F7AEE140E24993AA95E9F7E0
:10693400D4E0CAE8A6E1BEE14E8D4993BA95E1F7E9
:10694400AA95C9F7AEE1409138014993AA95E9F7B0
:106954004F91D8CFAB31B0F6B231A0F6AD5FAA2ECD
:10696400EF93FF934F925F926F927F9270F85F93D1
:10697400E42FF6EFB5E04424552466245527A4916A
:10698400A7FD539550FB40F8A6FD539550FB41F8E5
:10699400A5FD539550FB50F8A4FD539550FB51F8B9
:1069A400A3FD539550FB60F8A2FD539550FB61F88D
:1069B400F3955527A491A7FD539550FB42F8A6FDE6
:1069C400539550FB43F8A5FD539550FB52F8A4FD95
:1069D400539550FB53F8A3FD539550FB62F8A2FD69
:1069E400539550FB63F8F395442D37DE2196452DDE
:1069F40034DE2196462D31DE6C96BA9509F0BBCF74
:106A04005F9170FA7F906F905F904F90FF91EF913C
:106A140079CFFF93CF93DF936F937F93E42F6091AC
:106A2400190160FD1DC0F6EFD501DAE0C49136D03E
:106A3400B395AA2D96FD32D096FDB395F395AA2D64
:106A4400DA95A1F7AA2DAA5F96FDAA5FAA2E7F91D7
:106A54006F91DF91CF91FF91EF91BF91AF91089525
:106A6400F6E8EF77AE2FE0E8EA0FF21DAA0FEA0F7F
:106A7400F21DD501D6E0C49155D0B395AA2D96FD4B
:106A840051D096FDB395D0FD3196AA2DDA9599F79C
:106A9400AA2DAC5F96FDAC5FAA2ED9CF60913801C8
:106AA4006F936295C7FD629560933801A4D0A39556
:106AB40096FDA1D096FDA395C6FD6295609338011D
:106AC4009AD0A39596FD97D096FDA395C5FD6295A2
:106AD4006093380190D0A39596FD8DD096FDA39533
:106AE400C4FD62956093380186D0A39596FD83D04A
:106AF40096FDA395C3FD6295609338017CD0A39560
:106B040096FD79D096FDA395C2FD629560933801F8
:106B140072D0A39596FD6FD096FDA3956F91609367
:106B24003801089560913801D0FDC295762FC7FFD2
:106B34007295709338015FD0A39596FD5CD096FD55
:106B4400A395762FC6FF72957093380154D0A39500
:106B540096FD51D096FDA395762FC5FF729570933F
:106B6400380149D0A39596FD46D096FDA395762F7E
:106B7400C4FF7295709338013ED0A39596FD3BD027
:106B840096FDA3956093380108954F934591403045
:106B940011F44F91089567DEF9CFFF91EF91EE0F55
:106BA400FF1FAF93BF93B591BF3F11F0A5910ED0D6
:106BB400BF91AF914F934591403031F44F9131974C
:106BC400F695E795319609944EDEF5CFEF93E09173
:106BD4004A01E03039F0E730EF9111F40C9414726B
:106BE4005D010895EF91AE3108F0ADE1B73108F0E1
:106BF400B6E15D0108950F9300914A0107300F91AA
:106C040011F40C9415720E94B201D1E0C8ED6091A8
:106C140050016A1728F0609151016B1708F002C007
:106C24000C94AD0170914A01773069F0753031F000
:106C3400743041F0737039F0723008F43AC009F4DA
:106C440076C091C0A9C051E0AC3348F5BE3238F5E6
:106C5400B0FD550FB0FD550FA0FD550FB695A69587
:106C64006EE1B69FCA0FD21DC00DD11DA2EBB2E0DA
:106C7400CA0FDB1FA881B0913801BF70B295A07F05
:106C8400BA1779F0B0913801BF70AB2BA883A2EB8F
:106C9400B2E0CA1BDB0BB881B52BBF70B8830C9470
:106CA400AD01A2EBB2E0CA1BDB0BB8815095B52352
:106CB400F4CF6A2F6770639540E00894441F6A9587
:106CC400E9F7A695A695A695EA2F65E1F0914A0104
:106CD400F2FD60E1B69FCA0FD21DC00DD11DA09177
:106CE4003801F2FF08C0A695A170E9F44095A88187
:106CF400A423A883D4CF5E2FB695B695B695F5E1B7
:106D0400FB9FECE5FBE0E00DF11DE50FF21DA0910A
:106D14003801AF70508152955F705A1739F3508122
:106D2400507F5A2B5083A881A42BA883B8CF6A2FF5
:106D3400509138015695537043E0637031F0440F1D
:106D4400440F550F550F6A95C9F74095A695A6951A
:106D54006EE1B69FCA0FD21DC00DD11DA881A42318
:106D6400A52BA8839CCF6A2F509138015F7056954C
:106D740008F458604FE0617011F0429552954095C7
:106D8400A6956AE2B69FCA0FD21DC00DD11DA88177
:106D9400A423A52BA88383CF51E0AC33D0F4BE3217
:106DA400C0F4B0FD550FB0FD550FA0FD550FB695BD
:106DB400A6956EE1B69FD1E0C8EDCA0FD21DC00DF5
:106DC400D11DB0913801B27029F0B881B52BBF70D4
:106DD400B88365CFB8815095B523F9CFCE3108F08B
:106DE400CDE1EE3108F0EDE1D73108F0D6E1F7312D
:106DF40008F0F6E1EC1718F40E2EEC2FC02DFD1759
:106E040018F40F2EFD2FD02D0895EC1718F40E2E24
:106E1400EC2FC02DFD1718F40F2EFD2FD02D089543
:106E24000E94B201DBDF3F0140914A01403051F042
:106E3400443041F04130C9F5ACE5BBE0F0E875E120
:106E440060E106C0AAE8B4E0E8EDF1E07EE167E1C4
:106E5400C71758F5671648F5D61738F5761628F586
:106E64006C2F7D9FA00DB11DAC0FB21DE00DF11D67
:106E7400EC0FF21D0090380140E2572F5A955C0F39
:106E840056196C2F1EF0F7FF419302C00C90029428
:106E94000D92661511F06395F5CFA50FB21DE50FA0
:106EA400F21DD71511F0D395ECCF0C94AD010E94CF
:106EB400A2015F93AADFAC2FBD2F9DDEA395AE1771
:106EC400E1F799DEB395FB17E1F795DEAA95AC17C8
:106ED400E1F791DEBA95BD17E1F75F910C949B0140
:106EE4000E94A2015F9391DFBD2FAC2F84DEAE1709
:106EF40011F0A395FBCF7FDEFB1711F0B395F5CF0F
:106F04005F910C949B010E94B201E89489DF66DFD3
:106F14004C2FBD2FAC2FFDD052EF599351EFA395B9
:106F2400AE1711F05993FBCF53EF5993A42FB39598
:106F3400BF1739F0EED050EF5993AE2FEAD05993E2
:106F4400F5CFA42FE6D054EF599351EFA395AE1784
:106F540011F05993FBCF55EF59930C94AD01D3DF46
:106F64000E94B2013BDF5E2F5C1B515057FF09F4B6
:106F74000BC0FBEFECEE0AD0D395FDEFEFE006D0AB
:106F8400D395FEEEEDEE02D00C94AD01DE011EDED3
:106F94004F2F69DC652F4E2F66DC6A95E1F74F2F82
:106FA400439561CC0E94B201DE014FEFCE1B10F479
:106FB4004195C1955FEFDF1B10F45195D195CD1725
:106FC40060F000C06C2F669516DEAE1789F0A40F32
:106FD4006D1BD0F7B50F6C0FF7CF6D2F66950BDED9
:106FE400BF1731F0B50F6C1BD0F7A40F6D0FF7CF9F
:106FF4000C94AD01AF93AAEEA815F1F3A815F1F71F
:10700400AF9108950E94A201A0932901FBE8A6FD77
:10701400FCE8F0933B01AF73AA0FFDE8E0E8EA0F48
:10702400F21DA591A0932601A591A093270120927A
:10703400280120922401209225010C949B01209286
:107044002301409123014030E1F395C04F934091D7
:1070540022014030E1F74F9108955AD0A2EBCA0FB4
:10706400A2E0DA1FA881BA2FB295209223014091A1
:107074002301403041F440911C014B3110F4A883AA
:10708400F6CFB883F4CFA88376D042C03F933DEDCA
:1070940051D020922301409120014470431749F0BC
:1070A400403021F40E947F08342F03C00E94A008BE
:1070B400342F40912301403061F440911C014B3145
:1070C40020F448814F774883E6CF4881406848835D
:1070D400E2CF58815F7758833F910895D1E0C3EEA2
:1070E400CA0FD21D2092230140912301403061F444
:1070F40040911C014B3120F448814F774883F4CFF1
:10710400488140684883F0CF58815F775883089559
:10711400D501DEE1BD9FD1E0C8EDCA0FD21DC00D7F
:10712400D11D0895F6DF0F9302EBC00F02E0D01FCC
:107134000F910895D3E2BD9FD2E0C4E4CA0FD21DDB
:10714400C00DD11D0895BF934F930E94361CB42FD8
:107154004F91B0FF71F0BFEFB1B900001A99FECFA3
:1071640042B9B4E6BA95F1F72998B4E6BA95F1F7BD
:10717400299ABF9108950E94A2014F934091390129
:1071840041FD07C04F910C949B014F9144270C94EF
:107194009B014D7F40933901A0914A0140913501F3
:1071A40047FDA85F4A2F64D040911B015ED04091F7
:1071B4004C015BD0C0E0D1E0B0E14991429558D098
:1071C400BA95D9F76DD0C8EDD1E0A03031F4FEE224
:1071D400EEE155D0FA95E1F7D8CFA830D9F4F3E031
:1071E400E3E24DD0FA95E1F7E3E2F0913A01EF9F43
:1071F400C00DD11DF0E1E3E248814F77429538D0CC
:1072040049914F7735D0EA95B9F70E945239FA95EA
:1072140091F7BBCFA13031F4F3E8E5E130D0FA9532
:10722400E1F7B3CFA23031F4F4E5EEE128D0FA95DA
:10723400E1F7ABCFA33031F4FAE3EAE220D0FA95D8
:10724400E1F7A3CFA43011F4F7E5C2CFA53031F4B0
:10725400F0E4E0E114D0FA95E1F797CFA630A1F37A
:10726400A73011F40E94167290CF4295469547704C
:107274004F70405D4A3308F0495F0C946C39488183
:107284004295F6DF4991F4DFEA95C9F70C94523937
:10729400BF93B2E0A03009F0B064B4BDBF910895CB
:1072A400BF934F934DE0B0911801B6FD13D04AE05F
:1072B400B7FD10D04F91BF910895BF934F934DE008
:1072C400B0911801B6FD12D04AE0B7FD0FD04F912E
:1072D400BF910895BF93B0913101B030E1F740936D
:1072E4003201BA95B0933101BF910895609135018F
:1072F40064FF08955F935091C80055FFFCCF4093FD
:10730400CE005F910895BF93B0913301B030E1F79F
:10731400BA95B0933301B0913301B030E1F74091A5
:107324003401BF9108956091350164FFECCF409121
:10733400C80047FFFCCF4091CE000895609135010D
:1073440064FF0895EF93FF93BF93BA2FBB0FBE70F2
:10735400E0E7F3E7EB0FF21DB591B093CD00B591E3
:10736400B093CC00BF91FF91EF91089508230411CD
:1073740002080103008100500040002ABF93B0912D
:107384003301B030E1F7BA95B09333014091220153
:107394004D3E41F0B0913301B030C1F7409134011A
:1073A400BF9108954BE1BF9108956091350164FF49
:1073B400E5CF409122014D3EA9F34091C80047FF1B
:1073C400F8CF4091CE000895DF93CF93BF93AF934E
:1073D400FF93EF93CEE1D7E0E4E5F4E733D0EF9108
:1073E400FF91FF93EF93C7DECCE6D4E0B091200188
:1073F400B2FD7E9616F026D001C01ED04091220127
:10740400A1E04D3E69F0A2E0413F51F0A3E0423FCC
:1074140039F0A4E0433F21F0A5E0443F09F0DFCF79
:10742400B0912001B2FDAB5F4A2FEF91FF91AF9174
:10743400BF91CF91DF910895BEE1A191A993BA952F
:10744400E1F70895BEE1A591A993BA95E1F70895EE
:107454004E4E4E4E4E4EC0C0C0C0C0C080808080D4
:1074640080802E2E2E2E2E2E6E6E6E6E6E6EDF93FE
:10747400CF93BF93AF93FF93EF93CEE1D7E0E4E5CF
:10748400F4E7E0DFEF91FF91FF93EF93CCE6D4E0D4
:10749400D9DFCBCFACE5B0911801B3FDAFE5ACBDFE
:1074A400A1E1A093B800A0E0B4FFA1E0A093B900CB
:1074B4000895A82DA815F1F3A0912C01B0912B01EA
:1074C40008950E94B201A8EDB1E0C2EBD2E02D9282
:1074D4002197E9F740E050E00FD043954034D9F7C5
:1074E4000C94AD0167FF05C04F934C2FCD2FD42FC3
:1074F4004F917C2B660F0895E0E0F6EFF50FE40F53
:107504006491C0913801DC2FD295C07FD07FE3E035
:107514007727E8DF7295E6DF72957D93EA95C1F7E8
:1075240053955A3049F708950E94A2014F93A0E859
:10753400B7E0E0E0F6EFCAE0D0E845914D93DA9584
:10754400E1F7F096F096B096CA95B1F74F910C9486
:107554009B01FF93EF93BF70EFE0FDE8EB1BF49109
:10756400FF0FFA95F093520116F4F0935301EF9143
:10757400FF910895AF93A0913501A062A0933501C6
:10758400AF910895AF93A0913501AF7DF7CF0E94DD
:10759400B201AAE8B4E04EE15F73459FA00DB11DAE
:1075A400009038016093380155270E947E3A00927A
:1075B40038010C94AD010E94B201E42FF6EFA0E86B
:1075C400B7E05F77A50F5AE060E844914C93F395D8
:1075D400A60FB21D5A95C9F70C94AD010E94B201D1
:1075E4004F925F926F927F922F93C6E4D1E02C81E9
:1075F40048A05F846E84798859A16889A22FA370FA
:10760400E52F660FEE0FA33031F0660FEE0FA230B8
:1076140011F0660FEE0FF62FA0915801A13071F40E
:10762400E2013ED0803011F08FE133C0E30138D065
:10763400803011F080E22DC05CD02BC0A23091F4D8
:10764400E2012ED0803011F08FE123C0E30137D066
:10765400803011F082E11DC0ACE3BDE06A0E7B1EF8
:107664006CD017C0A33011F085E113C0A52DA33051
:1076740010F082E10EC0ACE3BDE04A0E5B1EF201E5
:1076840051916191E3010CD0803011F080E201C08E
:107694005ED02F917F906F905F904F900C94AD01CE
:1076A400CE0F10F48FE10895A0915001CA17D0F7BE
:1076B400DF0FC0F3B0915101DB17A0F70895659F68
:1076C400C00DD11D2296D33008F082E10895A22F77
:1076D4005091670160915601E52F660FEE0FA330BC
:1076E40031F0660FEE0FA23011F0660FEE0FF62F99
:1076F4000895571478F0D20134D0E8E8F1E064D06A
:10770400D3012FD0E8E8F1E084D0539473946A95C0
:1077140091F70895560E760E5A947A94D20121D098
:10772400E8E8F1E051D0D3011CD0E8E8F1E071D0F1
:107734005A947A946A9591F70895F3015193619359
:10774400D2010FD041D053946A95D1F70895F20134
:1077540051916191D30105D05CD073946A95D1F7AE
:1077640008956F93C8EDD1E0213011F465E103C0B1
:10777400253069F460E1B69FC00DD11D6A2F66956E
:1077840066956695C60FD21D4A2F6F9108952230D3
:1077940069F46EE1B69FC00DD11D6A2F669566959A
:1077A400C60FD21D4A2F440F6F9108956AE2B69F07
:1077B400C00DD11D6A2F66956695C60FD21D4A2F3E
:1077C400440F440F6F9108957F936F93BF93AF93CA
:1077D400652F742F777029F4A991A1936A95E1F725
:1077E4003FC0B0E8713019F0B6957A95FBCF772792
:1077F400A991AB9F703019F0A291A029A193119285
:1078040073957617A9F7A991AB9FA291A029A1938B
:1078140027C07F936F93BF93AF93652F742F7770B7
:1078240029F4A191A9936A95E1F71AC00F931F93C4
:107834000FEF11E0000F110F7A95E1F7652F7881B2
:10784400009570230095A191A19F072A0992712D9B
:107854006A95C9F768816023672B69930F911F911B
:10786400AF91BF916F917F9108950E94A2012E0163
:107874003F013FDF0C949B010E94A2012E013F01B6
:107884005CDF0C949B010E94A2012E013F015FDF8B
:107894000C949B010E94B20150E060E0FAE8EE27EC
:1078A400C0916701CF77D0915601DF7744914C9F07
:1078B400A12DE0954491E0954D9FB12DA51729F494
:1078C400B61719F4E39591F718C05A2F6B2FA091AE
:1078D4006601B0915501A50FB60F0E94FD35B61B88
:1078E400B61B0E94FD35A51BA51B0E94FD35B60FD6
:1078F400B60F0E94FD35E395C9F60C94AD010E94C4
:10790400B2016FEFFAE8EE27C0916701CF77D0910B
:107914005601DF7744914C9FA12DE0954491E09569
:107924004D9FB12DB61719F4E395A1F7E6CF5A2F61
:107934006B2FA0916601B09155017A2FB61BA51B40
:10794400750F0E94FD35B60FB60F0E94FD35B61BAC
:10795400B61BA3957A17A8F7E395E1F6CECFFF916E
:10796400EF911ED0EF93FF93409138014F93FF9313
:10797400EF9361D00E94CF350B09205052455353E9
:1079840020454E5445522000EF91FF914F91409372
:10799400380155DB4A3EE9F759DB0E94C01E0895C1
:1079A400EE0FFF1FC8E8D1E0459146954F9347700D
:1079B40049934F9142954770499358E145914993B2
:1079C400403011F05A95D1F729923197F695E79501
:1079D4003196C8E8D1E00895FF91EF91E1DFEF938C
:1079E400FF93409138014F93FF93EF9324D00E946B
:1079F400CF350B08202859296573202F20284E29BC
:107A04006F200000EF91FF914F914093380117DBF5
:107A1400493761F0493551F04E3619F04E3409F0CA
:107A2400F6CF14DB0E94C01E442708950FDB0E948A
:107A3400C01E41E00895FF93EF9392E02092360137
:107A4400A991B991B295B07FAF70AB0F0E94F43297
:107A5400DF93CF930E949E1EC2E0D8E0EBE1FCE0EE
:107A64000E948537A3E0B9E00E94E835CF91DF9109
:107A740058E14991403051F0DF93CF935F930E94D6
:107A840035345F91CF91DF915A9599F74091380140
:107A9400429540933801EF91FF9108950F931F93FE
:107AA4002F933F93A0935401B0935701C093660161
:107AB400D093550105D03F912F911F910F910895B7
:107AC4000E94A201B6D00E3118F4173108F415D073
:107AD400A0915401B0915701C0916601D091550114
:107AE400B983AA83AE3138F4B73128F435D0737032
:107AF400713009F06BD00C949B019BD0239F310F04
:107B04002596C00DD11DC00DD11D412FE8EDF1E02A
:107B14005EE1549FE00DF11DE00FF21D522F6991BB
:107B240061935A95E1F74395431781F740914A01D0
:107B3400463089F0412FEAE8F4E05EE1549FE00D1D
:107B4400F11DE00FF21D522F699161935A95E1F7EF
:107B54004395431781F708956CD0239F310F2596E1
:107B6400C00DD11DC00DD11D7727412FE8EDF1E0E7
:107B74005EE1549FE00DF11DE00FF21D522F619163
:107B840069936F7009F071E05A95C9F743954317EB
:107B940069F7E0916601F09155014081742B70837F
:107BA40040914A01463089F0412FEAE8F4E05EE171
:107BB400549FE00DF11DE00FF21D522F6191699366
:107BC4005A95E1F74395431781F7089532D0310F61
:107BD4002596412FE8EDF1E05EE1549FE00DF11DA3
:107BE400E00FF21D522F699161935A95E1F7439585
:107BF400431781F740914A014630D1F0412FEAE81A
:107C0400F4E05EE1549FE00DF11DE00FF21D522FF0
:107C14006991660F38F464FB60F96F70462E6081D9
:107C2400607F642961935A9599F74395431739F70F
:107C34000895C0916601D09155010A8119812C8162
:107C44003B8108950E94B201E0913801437001F52F
:107C5400A6E1B2E0C4E3D2E0F22D0BD0A0914A0138
:107C6400A63031F0A8ECB4E0C6EED4E0FE2F01D08B
:107C74006DC062E15AE149914D935A95E1F714962A
:107C840024966A95B9F75AE1FD935A95E9F7089550
:107C94004130E9F4ACE4B4E0CBE4D4E0F22D0BD011
:107CA400A0914A01A63031F0AEEFB6E0CDEFD6E0B8
:107CB400FE2F01D04BC063E159E14A914E935A958E
:107CC400E1F7FE93149725976A95B1F7089542302A
:107CD40001F5ACE4B4E0CEE2D4E0F22D0BD0A091F7
:107CE4004A01A63031F0AEEFB6E0C0EED6E0FE2F8A
:107CF40001D02CC062E15AE14A914E935A95E1F7C2
:107D0400149724976A95B9F75AE1FE935A95E9F7BF
:107D14000895A6E1B2E0C7E1D2E0F22D0BD0A09124
:107D24004A01A63031F0A8ECB4E0C9ECD4E0FE2F4F
:107D340001D00CC063E159E149914D935A95E1F7A3
:107D4400FD93259614966A95B1F708950C94AD01A8
:107D54004F935F937F9312DB4B3111F481E015C095
:107D64004130C9F7D0DA642FCEDA4095641711F0A8
:107D740084E20BC070E85527C6DA540F49937A950C
:107D8400D9F7C1DA451729F488277F915F914F917C
:107D9400089589E2FACF4F935F937F9341E09ADA93
:107DA400462F98DA409596DA70E855274991540F92
:107DB40091DA7A95D9F7452F8DDAE7CF0E94A2019F
:107DC40020923F01B0933F013092640130925D01F3
:107DD400C0935E01C0936001D0935F01D0936101B1
:107DE400E0936201F0936301A0935C01B0933F01BF
:107DF4000C949B010E94A201BA2FF8CFA0913F01DD
:107E040008955E984CE54093B80044E84093BC0064
:107E140044E94093BC00089544EA0EC05093BB006B
:107E240044E80AC044EC08D05091BB00089544E8EB
:107E340003D05091BB0008954093BC004091BC0016
:107E440047FFFCCF6091B900687F0895E5DF683093
:107E540089F4572F550F5E70506AE0DF683151F492
:107E64005B2FDCDF683231F45A2FD8DF683211F42B
:107E7400882708958FE05F915F91CACFE7DFCCDF59
:107E8400603169F4572F550F5E70516AC7DF603453
:107E940031F4CDDF683519F411968827B9CF8FE016
:107EA400B7CF052ED3DF502DB9DF683219F4119600
:107EB4008827AECF8FE00895AFDF6830A9F4572F3D
:107EC4005770550F5169AADF603471F4ABDF603528
:107ED40059F4A52FACDF683539F4BB27550FAA1F19
:107EE40008F4B095882794CF8FE092CF8827D830B4
:107EF40020F082E24F914F914FEF0895F7DFF99907
:107F0400FECFD2BDC1BDF89A40B521960895EEDFEB
:107F14008827F999FDCFD2BDC1BDF89A40B4441663
:107F240011F42196089540BDF894FA9AF99A789438
:107F3400F999FECFF89A219608954EBD4DB547FFA5
:107F4400FDCF4EB5089588272C9847EDF6DF4427DA
:107F5400F4DF2C9A4C7B4432B1F34C31A1F3483218
:107F640091F34C3281F3403371F3443361F3882746
:107F7400E894443A61F04C3951F06894483A39F045
:107F84004C3A29F0403B19F0443B09F081E1089553
:107F94008827D9DF803021F040E040939C10089579
:107FA4004C3911F448E0F9CF40E1F7CFF1DF40302C
:107FB40009F40895440F440F440F440F4A9508955B
:107FC400AA0FBB1F16F4AA0FBB1F4B2FB6DF4A2FF5
:107FD400B4DF422DB2DFB695A79516F4B695A795F2
:107FE4000895803059F44F93AEDF803031F42C98EB
:107FF40045E5A3DFE5DF2C9AA6DF4F910895803095
:1080040059F44F93A0DF803031F42C9843E595DF89
:10801400D7DF2C9A98DF4F910895803051F44F9315
:1080240092DF803029F42C9846E887DFC9DF2C9A48
:108034004F9108951196B0939D10A0939E1011979F
:10804400ECCF2FD2CEDF54D0E8CF7F93772710D058
:108054007F9108957F9371E00BD0D42F72E008D004
:10806400C42F7F9108957F9373E002D07F91089588
:108074008030C9F468DF8030B1F42C9842ED5DDFC4
:10808400AA0FBB1F16F4AA0FBB1FA3954B2F55DFD6
:108094004A2F53DF472F51DFB695A79516F4B695AF
:1080A400A79502D02C9A089548DF47DF46DF45DFC5
:1080B40044CF8030E1F447DF8030C9F42C9842ED9E
:1080C4003CDFAA0FBB1F16F4AA0FBB1F4B2F35DFD3
:1080D4004A2F33DF472F440F30DFB695A795B6F705
:1080E400B695A795E1DFD42F28DFC42F2C9A0895E5
:1080F4007F9370E010D07F9108957F9371E04D2FAE
:108104000AD072E04C2FB4DF7F9108957F9373E01F
:10811400AFDF7F9108958030A1F44F9314DF4F9126
:10812400803079F42C984F9347E807DF442705DF24
:1081340041E003DF472F01DF4F914F93FEDE2C9A7E
:108144004F910895803091F4FEDE8030D1F72C9861
:108154004F9347E8F2DE4427F0DE40E0EEDE472F9F
:10816400ECDE4F914F93E9DE2C9A4F9108958030C5
:10817400D1F4DF93CF934F935F93E5DE803079F4AE
:108184002C9847E8DADE4427D8DE4427D6DE40E0E0
:10819400D4DE55274991D1DE5A95E1F72C9A5F91A7
:1081A4004F91CF91DF9108958030B1F44F935F9355
:1081B400CADE803079F42C9847E8BFDE4427BDDE60
:1081C4004427BBDE40E0B9DE55274FEFB6DE5A95B3
:1081D400E1F72C9A5F914F9108958030E1F4DF9399
:1081E400CF934F935F93AFDE803089F42C9846EDA4
:1081F400A4DE4427A2DE4427A0DE40E09EDE44271E
:108204009CDE55279ADE49935A95E1F72C9A5F91A3
:108214004F91CF91DF910895BF93AF93DF93CF93A5
:108224004F935F937F93C0DF4FE062DF44276EDF9D
:10823400AA27BB27F2DE11964DEFCA2FCF70C130AB
:1082440009F44CEF55DF442761DFCC27DD2755DFE8
:10825400E4DE1196A03019F445EE0E9435344091C5
:108264009C10B41749F70AC0BF93AF93DF93CF9321
:108274004F935F937F938CDE403091F47F915F91B5
:108284004F91CF91DF91AF91BF910895B42FAA2759
:108294001197E9DEC42FBB27AA27E5DE4C1731F47A
:1082A400A0DEE1DE439532DFB8DEE8CF1196DBDEF7
:1082B4004C17E1F7F5CFDF93CF934F9392DE4DEF59
:1082C400CA2FCF70C13009F44CEF12DFC3DE219600
:1082D40014DF6ADFA2DE4F91CF91DF9108950E94EF
:1082E400A201AA27BB27ED0153DE4030A1F0F42FF1
:1082F400ACDE4C3F41F04D3F31F04B3A21F04F3072
:1083040018F0403908F421961196BF1789F740E018
:10831400DF1709F441E00C949B010F93BF93AF93D3
:108324004F93AA27BB27ED01FD0132DE403099F0BF
:10833400042F8BDE4D3F49F4DF93CF938BDE4D2F1B
:10834400CF91DF914F3F21F021964C3F09F43196B4
:108354001196B01771F74F91AF91BF910F91089596
:10836400FF93EF93DF93CF934F932F9311DE40301E
:10837400A9F0AA27BB2769DE242FB0919D10A091F4
:108384009E1040911401B41710F0A2E0BB27FD0128
:108394005CDE4D3F51F45EDED21738F42F914F91DD
:1083A400CF91DF91EF91FF910895159640919C1024
:1083B400B41709F4BB27BF1759F7AE1749F7AA2713
:1083C400BB270FDE42DE4F3F31F0405F242F90DEAB
:1083D40024DEDF01DDCFAFEFBFEFE0CF40937801C4
:1083E40050937A0160937C010895F8DF0E94B201F2
:1083F400CFDD403019F481E10C94AD0152D0B417B3
:1084040010F08BE1F9CF21DE4C3F11F087E1F4CF7E
:1084140040917A01403011F48BE1EECF413810F0F5
:108424008BE1EACF7ADFD03021F4C41710F488E16D
:10843400E3CFCCE3DFE050E06FEF69935A95E9F7BF
:10844400B3DE1196B0939D10A0939E1040917A01D3
:10845400CCE3DFE04F9384DFB993A9934BEA48DE82
:10846400DF93CF93F7DD219648DECF91DF91FBDDDB
:108474004DDEE0DDF9DE4F914A9561F712D0CCE391
:10848400DFE075DE40917C0133DEDF93CF93E2DDE4
:10849400219633DECF91DF91E6DD38DEBEDDACCF51
:1084A4009DDFA0917801A295BA2FA07FBF7011968D
:1084B400089594DF0E94B2017727F3DFC6DD4C3FB5
:1084C40069F0F7DDDF3F49F0BF93AF93DE01F3DEE0
:1084D400AF91BF91C9DE7F5FA1F7EDDE0C94AD01D2
:1084E4000E94A2014F935F937F932F93AA27BB27E8
:1084F4002ADDABDD242FD5DFA8DD4C3F39F489E13B
:108504002F917F915F914F910C949B0170917A010F
:10851400703810F08BE1F4CFCCDDDF3F11F48BE148
:10852400EFCFDE01CCE3DDE040917C01413009F482
:10853400D395423009F4DE5F1ADEDF93CF938ADDF0
:10854400D21759F02196D9DDCF91DF917EDDD0DDB0
:108554008ADDDCDD62DD88DED3CFADDE01DF7ADDEE
:108564002196CBDDCF91DF914BEAC2DD7CDDCEDD00
:1085740054DDED0196DF35DD70917A01770F4D2FD3
:10858400E1DD73954C2FDEDD60DDB2DD6CDDBEDD3B
:1085940044DDB6CF0E94A2014F935F937F9381DFA6
:1085A40054DD4C3F31F48EE17F915F914F910C94F7
:1085B4009B0170917A01703810F08BE1F5CF79DD71
:1085C400DF3F11F48BE1F0CFDE010BDDCCE3DDE026
:1085D40040917C01413009F4D395423009F4DE5FC7
:1085E400FCDDE2CF0E94A2014F935F937F9359DF9A
:1085F4002CDD4C3F11F48EE1D7CF77275ADDDE0115
:1086040070E0E8E8F1E055DDD193C19373957032E1
:10861400D1F7CACF0004080D11161A1F23282C30D5
:1086240035393D42464A4F53575B5F64686C7074FA
:10863400787C7F83878B8F92969A9DA1A4A7ABAEFB
:10864400B1B5B8BBBEC1C4C6C9CCCFD1D4D6D9DBB1
:10865400DDDFE2E4E6E8E9EBEDEEF0F2F3F4F6F761
:10866400F8F9FAFBFCFCFDFEFEFFFFFFFFFFFFFF36
:10868000000000CCC000333000FFF000000CCCCC68
:10869000CCCC333CCCFFFCCC000333CCC3333333E2
:1086A00033FFF333000FFFCCCFFF333FFFFFFFFF5C
:1086B000A5A5A506FF604E5440445E4024F4204228
:1086C000F240000000000000000000000000000078
:1086D000000000000EAE000004E000AAE800EE4E2C
:1086E000000000444040AA000066FF666842C4A241
:1086F00048A00000004400004888404222400A4A46
:108700000004E40000048000E000000040224880F3
:10871000EAAAE04C44E0E2E8E0E2E2E0AAE220E893
:10872000E2E0E8EAE0E24880EAEAE0EAE2E00404C3
:10873000000404802484200E0E00842480C268E497
:1087400000EEE04AAEA0CACAC0688860CAAAC0E803
:10875000C8E0E8C88068EA60AAEAA0E444E0E22A47
:1087600060AC8CA08888E0AEAAA0CAAAA04AAA40A1
:10877000EAE8804AAA60EAECA068E2C0E44440AAC1
:10878000AAE0AAAA40AAAEA0AA4AA0AA4440E248E7
:10879000E064446004A400C444C04A00000000E057
:1087A0004400004AAEA0CACAC0688860CAAAC0E82D
:1087B000C8E0E8C88068EA60AAEAA0E444E0E22AE7
:1087C00060AC8CA08888E0AEAAA0CAAAA04AAA4041
:1087D000EAE8804AAA60EAECA068E2C0E44440AA61
:1087E000AAE0AAAA40AAAEA0AA4AA0AA4440E24887
:1087F000E024C4204444448464808842208CEC807B
:1088000000F900F5F3F1F2FC00FAF8F6F4EB5E0083
:10881000F7000000007131000000797361773200C9
:108820000063786465343300002076667472350026
:10883000006E6268677A360000006D6A753738002E
:10884000002C6B696F303900002E2D6C00705C00BD
:1088500000000000002700000000EA2B00230000B9
:10886000003C00000000EC00003100343700000044
:10887000302C32353638ED00FB2B332D2A390000F1
:1088800000F900F5F3F1F2FC00FAF8F6F4EB000061
:10889000F700000000512100000059534157220009
:1088A00000435844452440000020564654522500B9
:1088B000004E4248475A260000004D4A552F2800D6
:1088C000003B4B494F3D2900003A5F4C00503F00B0
:1088D00000000000006000000000EA2A00270000FD
:1088E000003E00000000EC000031003437000000C2
:1088F00030E932353638ED00FB2B332D2A390000B4
:108900004400000000000000000000000000000023
:108910000000000000000000000000000000000057
:108920000000000000000000000000000000000047
:1089300000000000000000C000000000000000C1B6
:10894000000000000000000000002F0000000000F8
:1089500000000000000000000000EA000000C2006B
:10896000000000000000000000E100E2E000000064
:10897000E8E9E500E3E4ED00FB2BE72D2AE6000043
:1089800045000000000000000000000000000000A2
:108990000000000000400000000000000000000097
:1089A00000000000000000000000000000000000C7
:1089B000000000000000000000000000007B5B00E1
:1089C00000000000007D5D000000000000005C0071
:1089D00000000000000000000000007E0000000019
:1089E000007C00000000000000E100E2E000000068
:1089F000EFEEE500E3E4ED00FB2BE72D2AE60000B7
:108A0000FFFFFFFFFFFFFFFFFFFFFFFEFEFEFEFE7B
:108A1000FEFEFDFDFDFDFDFCFCFCFCFBFBFBFBFA93
:108A2000FAFAF9F9F9F8F8F8F7F7F6F6F6F5F5F4D1
:108A3000F4F3F3F2F2F2F1F0F0EFEFEEEEEDEDEC35
:108A4000EBEBEAEAE9E8E8E7E6E6E5E4E4E3E2E1BD
:108A5000E1E0DFDEDEDDDCDBDADAD9D8D7D6D5D46B
:108A6000D4D3D2D1D0CFCECDCCCBCAC9C9C8C7C63A
:108A7000C5C4C3C2C1BFBEBDBCBBBAB9B8B7B6B529
:108A8000B4B2B1B0AFAEADACAAA9A8A7A6A5A3A237
:108A9000A1A09E9D9C9B99989796949392918F8E5E
:108AA0008D8B8A898786858382817F7E7D7B7A789C
:108AB0007776747371706F6D6C6A696766656362EF
:108AC000605F5D5C5A595756545351504E4D4B4A56
:108AD0004847454442413F3E3C3B393836353332C6
:108AE000302E2D2B2A2827252422201F1D1C1A1941
:108AF00017161412110F0E0C0B09070604030100C0
:108B00000C11161A1E2225282B2D2F313233333407
:108B100034343434343434343535363738393B3CF6
:108B20003E40434547494B4D4F5152535454545482
:108B3000545351504E4C4A4745423F3D3A383634E3
:108B40003231302F2E2E2E2F303132333536383A07
:108B50003C3E4042444647494A4B4D4E4E4F505092
:108B60005050505050504F4E4D4C4B494846434149
:108B70003E3B37332F2B27221D18130D0802FDF81B
:108B8000F3EEE9E5E1DDDAD7D4D2D0CECDCCCCCB53
:108B9000CBCBCBCBCBCBCBCBCACAC9C8C7C6C4C344
:108BA000C1BFBCBAB8B6B4B2B0AEADACABABABAB98
:108BB000ABACAEAFB1B3B5B8BABDC0C2C5C7C9CB17
:108BC000CDCECFD0D1D1D1D0CFCECDCCCAC9C7C5D3
:108BD000C3C1BFBDBBB9B8B6B5B4B2B1B1B0AFAF28
:108BE000AFAFAFAFAFAFB0B1B2B3B4B6B7B9BCBE51
:108BF000C1C4C8CCD0D4D8DDE2E7ECF2F7FD02075F
:108C0000000A141D272F383F464B505457595959C5
:108C1000585654504C48433E39332E2925201C19B0
:108C200016141211111112131517191C1F222527C2
:108C30002A2C2E303132323232312F2D2B28252260
:108C40001F1C191613110F0D0C0B0A0A0A0B0C0E20
:108C500010121416181A1C1E1F2020201F1E1C196B
:108C600016120D0803FDF7F0EAE3DDD6D1CBC6C23C
:108C7000BFBDBBBABBBCBEC2C6CBD1D7DFE6EFF728
:108C80000008101920282E34393D41434445444200
:108C9000403D39342E29221C150F0802FCF7F2ED55
:108CA000E9E6E3E1E0DFDFDFE0E1E3E5E7E9EBED83
:108CB000EFF1F3F4F5F5F5F4F3F2F0EEECE9E6E3B9
:108CC000E0DDDAD7D4D2D0CECDCDCDCDCECFD1D37D
:108CD000D5D8DADDE0E3E6E8EAECEDEEEEEEEDEB3A
:108CE000E9E6E3DFDAD6D1CCC6C1BCB7B3AFABA9F6
:108CF000A7A6A6A6A8ABAFB4B9C0C7D0D8E2EBF57B
:108D000080675342352B221C16120E0C09070605EC
:108D1000040000000000000000000000000000004F
:108D2000807E7B79777572706E6C6A686664636149
:108D30005F5D5C5A5857555352504F4D4C4B494804
:108D40004745444341403F3E3D3C3B39383736354B
:108D50003433323231302F2E2D2C2B2B2A29282838
:108D60002726252524232322222120201F1F1E1DE4
:108D70001D1C1C1B1B1A1A19191818181717160076
:108D8000890091009A00A300AD00B700C200CE0098
:108D9000DA00E700F4000301120123013401460167
:108DA0005A016E0184019B01B301CD01E901060264
:108DB0002502450268028C02B302DC020803360376
:108DC00067039B03D2030C0449048B04D0041905E8
:108DD0006705B90510066C06CE063507A307170808
:108DE000930815099F09320ACD0A720B200CD80C82
:108DF0009C0D6B0E460F2F1025112A123F13641481
:108E0000F894A0E02A2EA1E03A2EA0E1AEBFAFEF89
:108E1000ADBFB0E0A0E0AA95F1F7BA95D9F7AAEBFB
:108E2000A4B9AFEFA5B9A0E8A7B9A0E0A8B9A0EF91
:108E3000AAB9AFEFABB9A6B1AF70A09335010E944C
:108E40000B790E940478B0FF5DC0B2ECB093800053
:108E5000B9E1B0938100F4E0A2FFF4E0F093870061
:108E6000FEEFA2FFF6EFF093860020928900FAE56C
:108E7000F0938800A2E0A0936F00A0E4A4BDA1E05D
:108E8000A5BDA1E3A7BD2092C000A0E1A093C100B1
:108E9000A6E6A093C200E8EAFFE87ED0A2E2B59180
:108EA000B993AA95E1F705B7036005BF0E7F05BF2B
:108EB0007894A8EC68D0B091C600B83719F0AA959C
:108EC000C9F720C0E8ECFFE867D045E140D0C8ED25
:108ED000D1E020D046E03BD0E0E0F0E0CCE3DFE0C2
:108EE00019D046E034D0CCEBDFE014D0FE3820F4CB
:108EF0000E9458793296789446E029D0AEEEB1E0DF
:108F00001BD0ECCFF89405B7016005BF0C7F05BFFF
:108F10000C94000028D0443039F446E018D0B091C9
:108F20003101B030E1F7EECF50E81DD01CD01BD09E
:108F300049935A95E1F717C04F2F429501D04F2F13
:108F40004F70405D4A3308F0495F4D930895BF93D9
:108F5000B0913101B030E1F740933201BA95B0934E
:108F60003101BF910895BF93B0913301B030E1F763
:108F7000BA95B0933301B0913301B030E1F740912D
:108F80003401BF910895AF93A82DA73EE9F3A82D12
:108F9000A73EE9F7AF910895C8EDD1E0A2E2B591FF
:108FA000B993AA95E1F708954156522D4368697027
:108FB00042617369633220284631313D55706461E6
:108FC0007465205379732920426F6F746C6F6164EC
:108FD0006572204572726F72202845534320746F6A
:088FE000206578697429202046
:10900000202020202020202020202020FFFFFFFFE4
:10901000FFFFFFFFFFFFFFFFFFFFFFFFFFFFFFFF60
:109C0000202020202020202020202020FFFFFFFFD8
:109C1000FFFFFFFFFFFFFFFFFFFFFFFFFFFFFFFF54
:10A80000202020202020202020202020FFFFFFFFCC
:10A81000FFFFFFFFFFFFFFFFFFFFFFFFFFFFFFFF48
:10B40000202020202020202020202020FFFFFFFFC0
:10B41000FFFFFFFFFFFFFFFFFFFFFFFFFFFFFFFF3C
:10C00000202020202020202020202020FFFFFFFFB4
:10C01000FFFFFFFFFFFFFFFFFFFFFFFFFFFFFFFF30
:10CC0000202020202020202020202020FFFFFFFFA8
:10CC1000FFFFFFFFFFFFFFFFFFFFFFFFFFFFFFFF24
:10D80000202020202020202020202020FFFFFFFF9C
:10D81000FFFFFFFFFFFFFFFFFFFFFFFFFFFFFFFF18
:10E40000202020202020202020202020FFFFFFFF90
:10E41000FFFFFFFFFFFFFFFFFFFFFFFFFFFFFFFF0C
:10F000000C94004700000000E0911801A0916501F8
:10F01000F9B1F3FBE5FFF1FBB0F9A7FFB3250895C4
:10F0200000000000000000000000000000000000E0
:10F03000000000004F935F936F93FF93EF93DF9374
:10F04000CF93BF93AF930F921F92FFB7FF93C4E18B
:10F05000D1E0B9A5B7FF5C98B7FD5C9AD5DFB9A739
:10F06000830C921CE9A1F92DF03029F4F82DFA3027
:10F0700010F1F63EF8F0FCE0E2FFFDEE8F1639F4F9
:10F080005E98E3FF17C0B2E8B093800013C0F1E1CF
:10F09000E2FFF3EF8F1639F45E9AE3FF0BC0B2EC98
:10F0A000B093800007C0F9E3E2FFF7E08F1611F498
:10F0B000882499242CC0A0918400A63EE0F3A73EAA
:10F0C00000F0A83E00F0A93E00F0AA3E00F0A8ED36
:10F0D000B1E0F6EFF80DC0E2ED91549140E060E848
:10F0E00048B9ED9156FD66B90000000055FD66B9BE
:10F0F000049054FD66B9CA95000053FD66B900003E
:10F10000000052FD66B9502D59F7000028B814D000
:10F11000E091C600E63711F40C948247FF91FFBFDF
:10F120001F900F90AF91BF91CF91DF91EF91FF9121
:10F130006F915F914F911895A0913D01E09133013E
:10F14000E03091F0EF3F21F4A0FD0EC0EEE30CC0E3
:10F15000EA95F5EFB491B5FF07C0B0913401B695CB
:10F16000A0FBB7F9B0933401E0933301E091310192
:10F17000E03091F0EF3F19F4E0E5AF770DC0EA958C
:10F18000F5EFB491B4FF08C0B0913201B0FB089420
:10F19000B795A7F9B0933201E0933101A0933D01F7
:10F1A0000895A0913D01E0913301E03091F0EF3FEF
:10F1B00021F4A0FD0EC0ECE70CC0EA95F5EFB49188
:10F1C000B7FF07C0B0913401B695A0FBB7F9B09373
:10F1D0003401E0933301E0913101E030E9F2EF3F97
:10F1E00019F4E0E9AF77D8CFEA95F5EFB491B6FF1F
:10F1F000D3CFB0913201B0FB0894B795A7F9B09383
:10F200003201CACF40911801C8EFD7E060D14091D8
:10F2100065015DD10895C8EFD7E051D14093180141
:10F220004ED1409365010895FF93EF93FBD0E09397
:10F230004001F0934101EF91FF910895E091400169
:10F24000F0914101A0E2A99FE00DF11DB096C0EB45
:10F25000D1E0A0E2B591B993AA95E1F7BFEFB993D8
:10F26000089547B740FDFDCFB7BFE89547B740FDCC
:10F27000FDCF089547B746FF0895B1E1F2DFFACF19
:10F28000F8944E2F407E19F4B3E0EBDFF3DFA0E1FA
:10F2900009901990B1E0E5DF3296AA95C9F7E03000
:10F2A00009F008953297B5E0DCDFE4DF3296089587
:10F2B000F8944F93BF93AF93B3E0D3DFDBDF329784
:10F2C000CCE3DFE0A0E8329609901990B1E0C9DF05
:10F2D000AA95C9F7B5E0C5DFCDDFAF91BF914F91DA
:10F2E0000895E0914001F0914101B097ACE0B591F3
:10F2F000B993AA95E1F7A0913501A7FD0895A6EA73
:10F30000B2E0CA0FDB1FACE0B0913801B993AA9507
:10F31000E9F70895E0E0F0E9A0E0BCE0492F4030D3
:10F3200029F3EA0FFB1F4A95FACF40914901477034
:10F33000AF93ECE0F0E9ACE0A49FF00D4491EE5FF8
:10F340005491EE50AF910895F8946AD0C0EBD1E09B
:10F35000A3EEB1E05CE04D9149935A95E1F742E4A8
:10F36000499353E140E2B9935A95E9F7A09788DFB2
:10F370009927B3E2B99FA4E4B2E0A00DB11DC8E89B
:10F38000D1E050E24D9149935A95E1F7299250E22C
:10F390004A91403219F428825A95D1F7C091E3017D
:10F3A000CF3519F4C8E8D1E004C00E941E00C0EBBC
:10F3B000D1E066DF93959F35E1F67894089530D0DB
:10F3C000A3EEB1E05CE045914D935A95E1F7749658
:10F3D000992750E2A0EBB1E045914D935A95E1F7A2
:10F3E000A8E8B1E040E253E24D935A95E9F7FF9364
:10F3F000EF939F930E9420009F91EF91FF91C8E8A7
:10F40000D1E0B3E2B99FA1E4B2E0A00DB11D53E297
:10F4100049914D935A95E1F793959F35D1F608950B
:10F420004091490147704295E0ECE49FE0E0F0E94B
:10F43000E00DF11D0895CCE3DFE04CE050E259937C
:10F440004A95E9F75FEF599343E150E259934A95A2
:10F45000E9F740EF5FEF59934A95E9F7E1DF28DFDD
:10F460003296CCE3DFE040E25FEF59934A95E9F74B
:10F470004BE04F931DDF32964F914A95D1F7789428
:10F480000895472F4770CEDFFF93EF93C9DFAF9109
:10F49000BF914CE04F93CCE3DFE040E055915993AE
:10F4A0004A95E1F7FF93EF93FD0102DF3296DF010A
:10F4B000EF91FF914F914A9569F778940895F999E2
:10F4C000FECFD2BDC1BDF89A40B521960895F999F5
:10F4D000FECFD2BDC1BD40BDF894FA9AF99A789496
:04F4E00021960895D4
:10F50000010101010101210101010101012181012B
:10F510000100002100110101010121D101010101BE
:10F520002101110101010121D1010101012101117B
:10F530000101010121D101010101010111010101BB
:10F540000101D1010101010101110101010101C10B
:10F55000010101010101010101000101C1010101DC
:10F56000010101010101010001C1010101010100CD
:10F57000010101010101410001010101010101003D
:10F58000000000400000000000000000000000003B
:10F59000000000000000000000000000000000006B
:10F5A000000000000000000000000000000000005B
:10F5B000000000000000000000000000000000004B
:10F5C000000000000000000000000000000000003B
:10F5D000000000000000000000000000000000002B
:10F5E000100000000000000000000000000000000B
:10F5F00020000000000000000000000000000000EB
:10F60000009010800090108000901080009010807A
:10F61000FC28288004C0145028282800000000007E
:10F6200000000000000000000000000000000000DA
:10F6300000000000000000000000000000000000CA
:10F6400000000000000000000000000000000000BA
:10F6500000000000000000000000000000000000AA
:10F66000000000000000000000000000000000009A
:10F67000000000000000000000000000000000008A
:10F6800028C004C0000000002088FC34B4000080C2
:10F690006400640064003C3C181818180000000066
:10F6A0000028000008A08080000004C028800024FA
:10F6B00028008000000044288000C004C418000016
:10F6C00000282828280028281818280000000000F2
:10F6D0008090808008A084408080C8A400004C8472
:10F6E00000000000000000008080601800802828D2
:10F6F000280000002828002828282800002CE8904E
:10F700000090108000901080009010800090108079
:10F710007C444480A8A814504844440024000000BD
:10F7200000183C3C185028280C3000000000000055
:10F73000241824400C401440242400000C003024E1
:10F7400024244424444040246424106460646424D9
:10F75000442444244064646464644048604818005D
:10F76000300060000400140060180C6028000000E5
:10F7700000000000300000000000000C1830000005
:10F7800028A004C02800002840847C6C5844A8802D
:10F79000003C003C003C18183C3C3C3C2400403001
:10F7A000182800001090808004C004C028FC287C29
:10F7B00028440C00000044EC8000C004C424000075
:10F7C00000282828286C2828C01828640000000079
:10F7D0008088A41010908440C004C8A400008C80CD
:10F7E000287C008080004084FCF8303000002448F1
:10F7F000280000002828002828282800002CE8C01D
:10F800000090108000901080009010800090108078
:10F81000FC44448080801450444444283C00000050
:10F8200000183C3C20546C181818181800000004EC
:10F830006428640C14603064646428281800186418
:10F84000646464646460606464180C6C605864642C
:10F8500064646464186464646464046060183C00F4
:10F860001800600004003400600000601800000010
:10F8700000000000300000000000001818180018F8
:10F88000449008A06C1C186C4084FC34B444A880DC
:10F8900024002400640000000000000064241830EC
:10F8A0002428282820888080A4A00C60448044401C
:10F8B00028440C40844444800000C0046C2400446C
:10F8C00000282828286C8080C018445440844810A0
:10F8D0008084BCB020888820D834C8A440848C8020
:10F8E0002C7C00C4C4448080C0082830008020885C
:10F8F000280000002828002828282800002CE8A03C
:10F900000090108000901080009010800090108077
:10F910007C808080808010908480804424186424BF
:10F9200000183C40780C7830300C7C180000000C3B
:10F93000681804183C44600C6464282830400C04A7
:10F94000046464606460606064180C78607C546473
:10F9500064646460186464643C640C60301864001F
:10F960000C2444242C2430207428146C185C742437
:10F970004824742448646464646440181818300C83
:10F98000448810906C34286C80807CD8EC6C6C803F
:10F990006424642464642424242424286060184893
:10F9A000404444442088408490A00C6044FC286477
:10F9B00080440C40844444280000C0046C2400802F
:10F9C00028444444446C80806018C44C600C18186F
:10F9D0008080BC1040848820E82CC8A480804C849F
:10F9E000EC2400C4EC448080C008144800802088C7
:10F9F000280000002828002828282800002CE8E4F7
:10FA00000090108000901080009010800090108076
:10FA1000FC808080B098109080ECEC44003C6464E2
:10FA20000018003C24183000300C2440004000181E
:10FA30007C180C0C6C044418242000006000040C9A
:10FA40002C6444606444447040180C50607C7C64B6
:10FA50004464442418646464183C18601818000056
:10FA6000000464606864486454180C78187C54641A
:10FA70006C6C5460306464643C640C30180C7C80A2
:10FA8000808410906C4040488080FC6CB46C6C802A
:10FA900064046464646464046404181824241830DE
:10FAA0001880442840844084808418308080282432
:10FAB00000440C40844444440000C00428241880BE
:10FAC0008080844080A800006018C480A008402482
:10FAD000A4B0BC4080808080E82CC8A488104084FA
:10FAE000E42428C4EC44D480C00814848080208896
:10FAF000288020882088808020888020882CE8F03A
:10FB00000000000090909090101010108080808075
:10FB10007C8080801090B098408080440040646475
:10FB2000001800401C307800300C7C182800003091
:10FB300054181804400464186404282830400C1831
:10FB40007C4064606460606464180C78606468641D
:10FB5000607C780418643C7C3C1830600C18000011
:10FB6000002064606440306464180C50187C646445
:10FB70006C6C602430646464182C181818180C0C11
:10FB800080842088C430286C80807CD8EC6C6C80A9
:10FB90004020646464646420642018180404183CE1
:10FBA00018008044408440848080301880FC801895
:10FBB00044448040844444440000C0042800244459
:10FBC0008080844080A800443018C480A00824406D
:10FBD000BCD0A41084404084E82CC8A44C8480800D
:10FBE000482428C4EC44F880C0081484808020880D
:10FBF000288020882088808020888020882CE82801
:10FC00000000000090909090101010108080808074
:10FC1000FC8080801090808084C4A8440000643CF4
:10FC20000000003C44686C00181818181800286080
:10FC3000641830640C646430640C281818001800D0
:10FC40007C6464646460606464186C6C60646464A4
:10FC500060686C6418643C7C641860600418000080
:10FC6000006464646460302064180C781864646410
:10FC7000482460043C683C7C3C0830181818001884
:10FC8000448820888018186C8080FC34B46C6C80A8
:10FC900064646464646840644064181864441818B8
:10FCA000400080804084208880843018DC80284098
:10FCB00000446040844444280000C0046C0024C414
:10FCC00044444444446C80443018C44C600C1818BC
:10FCD000BCB0808084402088E44CC4C44C848080C4
:10FCE000282400C4EC44D4D0FCF8148480002828D4
:10FCF000280028280000280028282820882CE83000
:10FD00000000000090909090101010108080808073
:10FD10007C4480441450808044EC442800004458C3
:10FD20000018003C18082C000C300000300028009F
:10FD3000242440240C242430242800300C003018C3
:10FD4000246444244440602464242864406464247B
:10FD5000602C642418241824641840480448004087
:10FD6000002044242424300464246C6C246464241F
:10FD7000600C6044182C183C6404400C18300000DF
:10FD8000449040842800004840847C6C58A84480FB
:10FD900064202424242C64206420242424000000D3
:10FDA000240080288080208890A0600CDCFC44180F
:10FDB00028446040844444EC0000C0046C002400EB
:10FDC00028002828286C804418184454408410487F
:10FDD000BCB0808080801090D094C0048C8040841F
:10FDE000284000C4C444FCF880802884800028286F
:10FDF000280028280000280028282820882CE830FF
:10FE00000000000090909090101010108080808072
:10FE1000FC4480441450A8A84080440000006000C6
:10FE200000000000000000000000000000000000D2
:10FE300000000000000000000000000000000000C2
:10FE400000000000000000000000000000000000B2
:10FE500000000000000000000000000000000000A2
:10FE60000000000000000024000028000000000046
:10FE700060080000000000000024000000000000F6
:10FE800028A08080000000604084FC34ECA84480FE
:10FE90000000000000000000000000001818181802
:10FEA0001800444480801090A4A0C004DC806C3C06
:10FEB00000446000004400800080C004C4002400AE
:10FEC00028002828286C282818182864000000001A
:10FED000A4B08080844008A0C8A480808C800000EA
:10FEE000444000808000D4F8408430480000282836
:10FEF000280028280000280028282824482CE8006A
:10FF00000000000090909090101010108080808071
:10FF10007C2880281450109080EC28000000C0003D
:10FF200000000000000000000000000000000000D1
:10FF300000000000000000000000000000000000C1
:10FF400000000000000000000000000000000000B1
:10FF500000000000000000000000000000000000A1
:10FF60000000000000000000000000000000000091
:10FF70000000000000000000000000000000000081
:10FF800028C080800000000020887CD858000080B5
:10FF900000000000000000000000000030303030A1
:10FFA00000004480808008A004C0C0048CFCA858D5
:10FFB00000006000004400280080C004C40000006D
:10FFC00028002828280028281818280000000000E9
:10FFD0008080000084400000C8A400004824000085
:10FFE00000000000000080800000600080002828E1
:10FFF000280028280000280028282828282CE80085
:00000001FF
